:04000000B9EF2BF039
:1000080000C01EF001C01DF002C01CF003C01BF0B0
:1000180004C01AF005C019F008C018F009C017F09C
:100028000AC016F00BC015F0E1CF27F0E2CF28F098
:10003800E9CF25F0EACF26F0F3CF23F0F4CF24F070
:10004800F5CF22F0F8CF1FF0F7CF20F0F6CF21F050
:100058004BEC28F022C0F5FF1FC0F8FF20C0F7FFC7
:1000680021C0F6FF23C0F3FF24C0F4FF1EC000F038
:100078001DC001F01CC002F01BC003F01AC004F040
:1000880019C005F018C008F017C009F016C00AF02A
:1000980015C00BF025C0E9FF26C0EAFF27C0E1FF25
:0600A80028C0E2FF110078
:1000AE000B6A0A6A096A00500402F4CF09F0F3CF12
:1000BE0008F001500502F4CF0BF0F3CF0AF0005018
:1000CE000502F3500926F4500A22E86A0B22015069
:1000DE000402F3500926F4500A22E86A0B2208C0E3
:1000EE0000F009C001F00AC002F00BC003F01200CC
:1000FE001E0E716E100E0001856F040E866F85C088
:10010E00E1FF86C0E2FFE69E85C0E1FF86C0E2FF0A
:10011E00E69C040E8525E16E000E8621E26EE68CCD
:10012E00180E456E040E466E45C0E1FF46C0E2FF56
:10013E00E69E45C0E1FF46C0E2FFE69C040E452464
:10014E00E16E000E4620E26EE68C020E8525E16E13
:10015E00000E8621E26E87C0E6FF88C0E6FF010E24
:10016E008525E16E000E8621E26E400EE66E85C09C
:10017E00E9FF86C0EAFFEECF00F085C0E1FF86C042
:10018E00E2FF400E0014E66E85C0E9FF86C0EAFF6E
:10019E00EECF00F085C0E1FF86C0E2FF880E0010B2
:1001AE00E66E85C080F086C081F0040E8519006E63
:0601BE0000C085F01200F4
:1001C4000B820BAEECEF00F0036802680168006874
:0801D4000A360232FF0E120090
:1001DC000B840BAEF9EF00F0010E036E026A016A9C
:0A01EC00006A0A360232FF0E12000C
:0801F6000AAE029E000E120089
:1001FE000401286B296B47D004013D8E2881000134
:10020E007F51010A02E10401288352D03D8E50D065
:10021E0004013D8E24BF16D024C403F00F0E031626
:10022E0003C000F0000E016E003600900136830E02
:10023E000024E96E000E0120EA6EEECF04F0EECF40
:10024E0005F015D024C403F00F0E031603C000F002
:10025E00000E016E003600900136430E0024E96E4A
:10026E00000E0120EA6EEECF04F0EECF05F004C0D2
:10027E00E9FF05C0EAFFEECF01F001A403D00401AF
:10028E00010E286F15D020C401F01F0E011601506B
:10029E00000AB2E020C401F01F0E01160150010A3F
:1002AE00B5E020C401F01F0E01160150020AB0E0A5
:1002BE003DAE07D0280E3A6E040E3B6E3D80020E08
:0402CE003E6E12006E
:0E02D200026A016A006A086A036A000E1200DE
:1002E0003D8E716A426A22C439F03950000A03E136
:0E02F000100E386E03D0200E386E01DF1200A3
:1002FE0004012051800AD8A473D0C00E3D6E65D083
:10030E00000E006E5C0E016E000E026E00C03AF022
:10031E0001C03BF002C03CF0120E3E6E000E3F6E6E
:10032E005FD0030E006E000E016E22C404F0000EAC
:10033E00056EB6DE6C0E0024E96E000E0120EA6E2C
:10034E00EECF3AF0EECF3BF0EECF3CF0020E3A2479
:10035E00F66E000E3B20F76E000E3C20F86E090084
:10036E00F5CF00F00900F5CF01F000C03EF001C05E
:10037E003FF036D022510001825D23E3030E006E62
:10038E00000E016E22C404F0000E056E89DE470ECB
:10039E000024E96E000E0120EA6EEECF3AF0EECFA9
:1003AE003BF0EECF3CF03AC0F6FF3BC0F7FF3CC04F
:1003BE00F8FF0900F5CF00F000C03EF0000E3F6ED2
:1003CE0001D03D6A0DD03D6A0BD004012351010AC4
:1003DE0097E02351020AA5E02351030ACBE0F3D79D
:0203EE001200FB
:1003F00020C401F01F0E01160150010A01E08DD04A
:1004000004012451000A01E088D02151060A3FE18D
:1004100034D03950010A17E1FE0E006E5A0E016EFB
:10042000000E026E120E0026000E0122022200C0F3
:100430003AF001C03BF002C03CF0090E3E6E000EE7
:100440003F6EC00E3D6E23D03950010A12E1950E69
:10045000006E5B0E016E000E026E00C03AF001C02D
:100460003BF002C03CF0210E3E6E000E3F6EC00E0F
:100470003D6E0DD0800E3D6E0AD004012351210A3D
:10048000C8E02351220AE0E02351230AF3E020C40C
:1004900001F0600E0116050E006E005004E00132FE
:1004A000019EFF0FFBD70150010A01E036D022D098
:1004B00034D033D0750E3A6E000E3B6E010E3E6E98
:1004C000000E3F6EC10E3D6E28D0800E3D6E23C4DF
:1004D00075F023D0710E3A6E000E3B6E010E3E6E2B
:1004E000000E3F6E810E3D6E18D0800E3D6E22C410
:1004F00071F013D004012151010ADAE02151090AF7
:10050000D8E02151020AD6E021510A0ADEE0215149
:0C051000030AE0E021510B0AE8E01200B1
:10051C0004012251010A11E120C401F01F0E011641
:10052C000150000A0AE13D8E2151030A04E1010E3B
:10053C0000017F6F02D000017F6B04012251000A81
:10054C00D8A48BD020C401F01F0E01160150020A52
:10055C00D8A483D024C401F00F0E01160150000A58
:10056C00D8B47BD03D8E24BF16D024C403F00F0E1C
:10057C00031603C000F0000E016E00360090013629
:10058C00830E0024E96E000E0120EA6EEECF04F01B
:10059C00EECF05F015D024C403F00F0E031603C0E4
:1005AC0000F0000E016E003600900136430E002460
:1005BC00E96E000E0120EA6EEECF04F0EECF05F0EE
:1005CC002151030A07E104C0E1FF05C0E2FF840EDC
:1005DC00E66E43D024C400F00F0E0016700E026EAF
:1005EC000F0E036E00500226D8B0032A02C0E9FF9A
:1005FC0003C0EAFFFE0EEE14006EEECF01F0FF0E0C
:10060C00011602C0E1FF03C0E2FF00C0E6FF01C01B
:10061C00E6FF24AF11D004C0E1FF05C0E2FFE66A9B
:10062C00040E0418006E00C004F004C0E1FF05C005
:10063C00E2FF400EE66E11D004C0E1FF05C0E2FF00
:10064C00880EE66E040E0418006E00C004F004C0A0
:0C065C00E1FF05C0E2FFC80EE66E1200D0
:10066800000E3F5C02E1080E3E5C10E23EC003F063
:100678003FC004F04050000A03E1010E406E05D06F
:100688004050010A02E1020E406E04D0080E036ECB
:10069800000E046E43C0E1FF44C0E2FFE69243C08F
:1006A800E1FF44C0E2FFE69043C0E9FF44C0EAFF2F
:1006B800EECF00F043C0E1FF44C0E2FF0450001059
:1006C800E66E010E4324E16E000E4420E26E03C084
:1006D800E6FF03503E5C006E04503F58016E00C0B8
:1006E8003EF001C03FF0280E0001896F040E8A6FAA
:1006F8003DB02FD0035004102BE03AC0F6FF3BC0AA
:10070800F7FF3CC0F8FF0900F5CF00F089C0E1FF12
:100718008AC0E2FF00C0E6FF894B8A2B010E3A240B
:10072800006E000E3B20016E000E3C20026E00C0E1
:100738003AF001C03BF002C03CF0010E035C006ED1
:10074800000E0458016E00C003F001C004F0D2D7B7
:1007580024D00350041021E03AC0E9FF3BC0EAFF6F
:1007680089C0E1FF8AC0E2FFEECFE6FF894B8A2B02
:10077800010E3A24006E000E3B20016E00C03AF0D4
:1007880001C03BF0010E035C006E000E0458016EC0
:0C07980000C003F001C004F0DCD7120028
:1007A400010E00016F25E96E000E7021EA6EEECF96
:1007B40000F000C002F0000E8F5D02E102508E5D79
:1007C40003E28EC002F00AD002508E5D006E000E6D
:1007D4008F59016E00C08EF001C08FF0036A025081
:1007E400035C1CE2280EE96E040EEA6E0350E9264F
:1007F400D8B0EA2AEECF00F08BC0E1FF8CC0E2FF54
:1008040000C0E6FF010E8B25006E000E8C21016EE8
:1008140000C08BF001C08CF0032AE1D7000E006EFB
:100824008F51005C02E18E51000828E2010E9525EB
:10083400E16E000E9621E26E080EE66E020E95251C
:10084400E16E000E9621E26E280EE66E040EE66E50
:100854006FC0E9FF70C0EAFFEECF00F000BC07D024
:1008640095C0E1FF96C0E2FFC80EE66E06D095C0C3
:10087400E1FF96C0E2FF880EE66E19D0010E9525C1
:10088400E16E000E9621E26E080EE66E020E9525CC
:10089400E16E000E9621E26E200EE66E040EE66E08
:1008A40095C0E1FF96C0E2FF840EE66E8D9F1200B4
:0A08B4000001745301E09ADD120008
:1008BE000CB0A1EF04F00CA249EF05F00E6A000E89
:1008CE000264B8EF04F0F00E0214D8A483EF04F023
:1008DE00023A01380F0B02260138F00B016E003878
:1008EE000F0B01260038F00B006E08380F0B002698
:1008FE000838F00B086E0E84D89002BE9CEF04F000
:10090E0008360036013602360E2A02BE9CEF04F07F
:10091E0008360036013602360E2A02BE9CEF04F06F
:10092E0008360036013602360E2A0E5003643DEFAD
:10093E0005F0035E0BBC08AE43EF05F0D880800EC9
:10094E0008640030000E002201220222D8A043EFDC
:10095E0005F0023201320032034A49EF05F043EF4F
:10096E0005F001C002F000C001F008C000F0086AF6
:10097E00000E0E860264EFEF04F0F00E0214D8A4FF
:10098E00D7EF04F0023A01380F0B02260138F00BB4
:10099E00016E00380F0B01260038F00B006E0E842E
:1009AE00D89002BE9CEF04F00036013602360E2AB5
:1009BE0002BE9CEF04F00036013602360E2A02BE4D
:1009CE009CEF04F00036013602360E2A9CEF04F03E
:1009DE0001C002F000C001F0006A000E0E960E88F3
:1009EE0002641CEF05F0F00E0214D8A407EF05F018
:1009FE00023A01380F0B02260138F00B016E0E84FD
:100A0E00D89002BE9CEF04F0013602360E2A02BECA
:100A1E009CEF04F0013602360E2A02BE9CEF04F063
:100A2E00013602360E2A9CEF04F001C002F0016A74
:100A3E00000E0E8602644FEF05F0F00E0214D8A4DD
:100A4E002BEF05F0023A0E84D89002BE9CEF04F014
:100A5E0002360E2A02BE9CEF04F002360E2A02BEA9
:100A6E009CEF04F002360E2A9CEF04F0010E0C6E81
:100A7E00EEEC00F052EF05F0020E0C6EFBEC00F007
:100A8E0052EF05F0040E0C6EE2EC00F052EF05F0A2
:080A9E00080E0C6E17DC1200BB
:100AA600416A43C0E1FF44C0E2FFE66A040E431810
:100AB600E16E44C0E2FF000EE21AE66A00018DAF65
:060AC60001D08D9F12001B
:100ACC006D983DBE4AD000018DAF28D0020E416E0C
:100ADC00010E4324E16E000E4420E26EE66A43C030
:100AEC00E1FF44C0E2FFC80EE66E010E9525E16EF3
:100AFC00000E9621E26E080EE66E020E9525E16E52
:100B0C00000E9621E26E280EE66E040EE66E95C07F
:100B1C00E1FF96C0E2FFC80EE66E1ED0010E9525D1
:100B2C00E16E000E9621E26E080EE66E020E952521
:100B3C00E16E000E9621E26E200EE66E040EE66E5D
:100B4C0095C0E1FF96C0E2FF8C0EE66E43C0E1FF5C
:100B5C0044C0E2FF840EE66E80D000018DBF7DD0D4
:100B6C00040120AF52D03F50275D02E13E50265D7C
:100B7C0004E226C43EF027C43FF070DD010E416E46
:100B8C00010E00019525E16E000E9621E26E080E15
:100B9C00E66E020E9525E16E000E9621E26E200E99
:100BAC00E66E040EE66E95C0E1FF96C0E2FF800E85
:100BBC00E66E946B010E6F25E16E000E7021E26EF5
:100BCC00080EE66E020E6F25E16E000E7021E26ECD
:100BDC00200EE66E040EE66E6FC0E1FF70C0E2FF01
:100BEC00840EE66E010E946F020E4324E16E000E2D
:100BFC004420E26E280EE66E040EE66E43C0E1FF62
:100C0C0044C0E2FFC80EE66E28D00001020E416E11
:100C1C00010E4324E16E000E4420E26EE66A43C0EE
:100C2C00E1FF44C0E2FFC80EE66E010E9525E16EB1
:100C3C00000E9621E26E080EE66E020E9525E16E10
:100C4C00000E9621E26E280EE66E040EE66E95C03E
:0C0C5C00E1FF96C0E2FFC80EE66E120039
:100C680020C401F0600E0116050E006E005004E06D
:100C78000132019EFF0FFBD70150000A01E05CD052
:100C880038D03D8E080E386E57D07FEC01F054D026
:100C980070EC01F051D0390E3A6E000E3B6E3D807B
:100CA800010E3E6E3D8E48D0FFEC00F045D032DCA0
:100CB80043D0420E006E000E016E0401245100263E
:100CC800D8B0012A00C03AF001C03BF03D80010EC7
:100CD8003E6E3D8E31D03D8E420EE16E000EE26ECC
:100CE8002451E126D8B0E22A22C4E6FF25D024D038
:100CF80023D004012151050AC4E02151060AC5E0A8
:100D08002151090AC5E02151080AC5E02151000A0C
:100D1800CBE02151010ACBE02151030AC8E021515F
:100D28000A0AC7E021510B0AD6E02151070ADFE081
:0A0D380021510C0ADDE0DCD71200A7
:100D4200FE0E00016C6F5A0E6D6F000E6E6F430E39
:100D5200476E5C0E486E000E496E730E4A6E5B0E55
:100D62004B6E000E4C6E9E0E4D6E5A0E4E6E000E67
:040D72004F6E1200AE
:0E0D7600160E6F6E9F0E6B6E3B0E696E1200B6
:100D84006D92699468A403D0FB0E6816FBD7120019
:100D94004150020A02E104DD1ED083DE9451000AB0
:100DA40019E1010E9525E16E000E9621E26E080E02
:100DB400E66E020E9525E16E000E9621E26E200E7F
:100DC400E66E040EE66E95C0E1FF96C0E2FF8C0E5F
:080DD400E66E01D0946B1200E1
:100DDC0043C0E9FF44C0EAFFEECF00F000AE05D0FF
:100DEC0043C0E1FF44C0E2FFE66A406A416A3E6AE2
:0C0DFC003F6A3D6A33DF58DD63DE120001
:040E0800A19A120099
:100E0C000B800BAE12EF07F0026A0AAEFF0E026EF9
:0C0E1C00016E006E0A360232FF0E12005A
:100E28000D6A086A0050D8B4000C04180A6E0ABE8D
:100E38000D1E0B6A04AE02D0041E042A00AE02D0B6
:100E4800001E002A005004100A6E0ABE1FD004506B
:100E5800085E003600340836045008260036060EB0
:100E68000C6E00340836045000B0085E00A0082656
:100E780000360C2EF6D700A008260BB015D00DAE04
:100E8800000C001E002A081E082A000C04AE09D017
:100E980000BE04D00050086E006AF1D7006A002A2C
:100EA800000C001E0B2AD3D7082A0450085CD8A4CB
:0E0EB800E6D7086A002A00AEE2D7FF0C12004F
:100EC60070A019D06FC0E9FF70C0EAFFEECF01F045
:100ED6000150800A0FE143C0E9FF44C0EAFFEECFAC
:100EE60001F00150840A06E16FC0E1FF70C0E2FF25
:0C0EF6008C0EE66E7090DF0E6816120085
:100F0200040E4318006E00C043F03850080A0AE18C
:100F120022C46EFF6E50000803E2100E386E02D03B
:100F2200040E386E4150010A3BE1020E4324E16E89
:100F3200000E4420E26E280EE66E040EE66E34ECDD
:100F420003F04050020A07E143C0E1FF44C0E2FF60
:100F5200840EE66E24D0040E4318006E00C043F0E7
:100F620043C0E9FF44C0EAFFEECF00F000BC0CD062
:100F7200040E4318006E00C043F043C0E1FF44C0BA
:100F8200E2FFC80EE66E0BD0040E4318006E00C0DE
:100F920043F043C0E1FF44C0E2FF880EE66E01D099
:040FA20081DD1200DB
:0A0FA6006984EF0E68166D821200D8
:100FB000086A080E0C6E003408360450085ED8B07B
:0E0FC00002D00826D89000360C2EF5D712006D
:080FCE000B6A0B86FF0E1200F6
:100FD600025006180E6E086A096A0B6A0350076407
:100FE600DEEF08F006500A6E068E028E03500B6E78
:100FF6000750036E000E0B642EEF08F00B50075ED1
:10100600D8B4CFEF08F0070E07649DEF08F0075E2F
:1010160000C008F001C000F002C001F0026A074EED
:10102600CFEF08F0076472EF08F0075E00C008F023
:1010360001C000F0016A074ECFEF08F0076450EFD9
:1010460008F0075E00C008F0006A074ECFEF08F010
:10105600076437EF08F00AC002F005C001F004C0CB
:1010660000F0086AFBEF09F0030E076442EF08F090
:10107600075E08380F0B086E074ECFEF08F0D890C2
:101086000832074ECFEF08F0D8900832074ECFEF60
:1010960008F0D8900832CFEF08F0030E076461EF2E
:1010A60008F0075E08380F0B086E0038F00B0826AC
:1010B60000380F0B006E074ECFEF08F0D8900032C5
:1010C6000832074ECFEF08F0D89000320832074EAC
:1010D600CFEF08F0D89000320832CFEF08F0030EB9
:1010E600076489EF08F0075E08380F0B086E0038B2
:1010F600F00B082600380F0B006E0138F00B0026A7
:1011060001380F0B016E074ECFEF08F0D890013271
:1011160000320832074ECFEF08F0D8900132003285
:101126000832074ECFEF08F0D8900132003208326D
:10113600CFEF08F0030E0764BAEF08F0075E083831
:101146000F0B086E0038F00B082600380F0B006EE8
:101156000138F00B002601380F0B016E0238F00B38
:10116600012602380F0B026E074ECFEF08F0D8901B
:101176000232013200320832074ECFEF08F0D89023
:101186000232013200320832074ECFEF08F0D89013
:101196000232013200320832096A000E0EAEC3EF87
:1011A60009F0081E001E011E021E082A0022012246
:1011B6000222C3EF09F00750D8A4E4EF08F0FBEFD2
:1011C60009F0096A02C00AF0028E068E0750035C17
:1011D600076ED8B4B6EF09F0070E076484EF09F07E
:1011E600075E0450096E0550046E0650056E066AC9
:1011F600074EB6EF09F0070E076459EF09F0075ED0
:101206000450096E0550046E056A074EB6EF09F0E4
:10121600070E076437EF09F0075E0450096E046A8B
:10122600074EB6EF09F0070E07641EEF09F00AC075
:1012360002F0FBEF09F0030E076429EF09F0075EE1
:1012460009380F0B096E074EB6EF09F0D890093230
:10125600074EB6EF09F0D8900932074EB6EF09F0FF
:10126600D8900932B6EF09F0030E076448EF09F08B
:10127600075E09380F0B096E0438F00B092604388F
:101286000F0B046E074EB6EF09F0D8900432093200
:10129600074EB6EF09F0D89004320932074EB6EF82
:1012A60009F0D89004320932B6EF09F0030E07644C
:1012B60070EF09F0075E09380F0B096E0438F00B62
:1012C600092604380F0B046E0538F00B0426053882
:1012D6000F0B056E074EB6EF09F0D89005320432B3
:1012E6000932074EB6EF09F0D890053204320932BA
:1012F600074EB6EF09F0D890053204320932B6EF40
:1013060009F0030E0764A1EF09F0075E09380F0B19
:10131600096E0438F00B092604380F0B046E0538E5
:10132600F00B042605380F0B056E0638F00B052664
:1013360006380F0B066E074EB6EF09F0D890063248
:10134600053204320932074EB6EF09F0D89006325C
:10135600053204320932074EB6EF09F0D89006324C
:10136600053204320932086A000E0EAEC3EF09F0E8
:10137600091E041E051E061E092A0422052206222F
:101386000950082604500022055001220650022268
:101396000EBEDAEF09F0D8A0E9EF09F00232013209
:1013A60000320832033EE9EF09F0F5EF09F0D8B054
:1013B600EFEF09F0000E081E001E011E021E082A8D
:1013C6000022012202220A7EEFEF09F0010E0C6EC6
:1013D6005FEC04F0FDEF09F0020E0C6E5FEC04F01A
:1013E600FDEF09F0040E0C6EE2EC00F0FDEF09F0E3
:0613F600000E0C6E120057
:1013FC00A2DC806B816B7B6B7C6B6A6A686AB5DC88
:10140C006D8C6E6A716A6D9C7D6B7E6B000E7E5D61
:10141C0002E1080E7D5D17E27DC000F07EC001F098
:10142C00003600900136003600900136000E002484
:10143C00E16E040E0120E26EE66AE66AE66AE66A8E
:10144C007D4B7E2BE3D7160E706E68A603D0F70E7D
:10145C006816FBD73D6A8D6B8E6B8F6B6D98080E83
:0C146C00436E040E446E396A386A1200A8
:101478000134083609360450085E0550D8A0053CEA
:10148800095E003601360F0E0C6E01340836093637
:10149800045000A006D0085E0550D8A0053C095E9F
:1014A80005D008260550D8B0053C09260036013677
:1014B8000C2EEBD700B006D0045008260550D8B043
:0814C800053C0926000012009A
:1014D000086A096A000E07620364EDEF0AF0025021
:1014E00006180A6E075003267E0ED8A07EEF0AF07B
:1014F000035ED8B0F2EF0AF082EF0AF0035ED8A0E4
:10150000F7EF0AF0028E068E02C00EF001C00BF05B
:1015100000C00DF000500402F4CF0CF001500502A1
:10152000F4CF00F0F3CF08F00402F3500C26F4508F
:101530000822000E00220D500502F3500C26F45034
:101540000822000E002202500402F3500826F45034
:10155000002202500502016A000E0122F35000260B
:10156000F45001220D500602F3500826F4500022D8
:10157000026A000E012202220B500602F3500026DE
:10158000F4500122000E02220E500602F3500126F2
:10159000F450022202BED5EF0AF0083600360136BA
:1015A00002360306D8B4F7EF0AF0E8EF0AF0D88065
:1015B000800E08640030000E002201220222D8A012
:1015C000E8EF0AF0023201320032034AF2EF0AF089
:1015D0000AAE029E000EFAEF0AF0010E69EC01F06D
:1015E000FAEF0AF0020EE2EC00F0FAEF0AF0040E55
:0615F000EEEC00F0120019
:0615F600067EEEDC12008F
:1015FC000001D751390806E3300ED75D03E3010E25
:08160C00006E01D0006A12001B
:101614000A6A0350D8A40A800750D8A40A820A5040
:10162400D8B46DEF0BF0030AD8B426EF0BF00AB070
:1016340021EF0BF006AE6BEF0BF069EF0BF002AE8F
:1016440069EF0BF06BEF0BF00250800B0A6E029EF9
:101654000650800B069E0A18D8B437EF0BF00A50D8
:10166400D8B469EF0BF06BEF0BF00750035CD8B400
:1016740041EF0BF0D8A05DEF0BF063EF0BF00650D9
:10168400025CD8B44BEF0BF0D8A05DEF0BF063EF26
:101694000BF00550015CD8B455EF0BF0D8A05DEF0A
:1016A4000BF063EF0BF00450005CD8B46DEF0BF05B
:1016B400D8B063EF0BF00A52D8B46BEF0BF069EFBC
:1016C4000BF00A52D8B469EF0BF06BEF0BF0D88033
:0E16D4001200D8901200D880D88412001200A4
:1016E2000450000A12E10550000A0FE10650000AF8
:1016F2000CE10750000A09E1FF0E006EFF0E016EB9
:101702007F0E026EFF0E036EA8D0086A096A0750A8
:10171200D8B41CEF0CF00350D8B421EF0CF00250F7
:1017220006180A6E028E068E0E6A02C008F001C00A
:101732000CF000C00DF004500D5E0550D8A0053C21
:101742000C5E0650D8A0063C085E086A0C6A0D6A58
:10175200D8A0B3EF0BF0D890023201320032083237
:10176200010E0E6E0750035ED8A0C0EF0BF07E0E86
:101772000E240326D8B026EF0CF0C6EF0BF07E0E37
:101782000E240326D8A02BEF0CF0180E0B6E0D368C
:101792000C3608360036013602360E360450005E2C
:1017A2000550D8A0053C015E0650D8A0063C025E5A
:1017B20006340E120EA0E1EF0BF00D80ECEF0BF0F1
:1017C200045000260550D8B0053C01260650D8B07A
:1017D200062802260D900B2EC8EF0BF012EF0CF02C
:1017E200D8900036013602360E360450005E05509F
:1017F200D8A0053C015E0650D8A0063C025E063425
:101802000E10010B0D26D8B00C2AD8B4082AD8A481
:1018120012EF0CF008320C320D32032AD8B426EF44
:101822000CF00AAE089E0850026E0C50016E0D506C
:10183200006E2EEF0CF0010EE7EC07F02EEF0CF02D
:10184200020E69EC01F02EEF0CF0040EE2EC00F057
:0C1852002EEF0CF0080EEEEC00F012007F
:10185E003850000A0AE16D6A696ABBEC06F06DB693
:10186E0002D06D86FCD7010E386E3850010A08E1A1
:10187E006DBA06D0686A696A69806988020E386E28
:10188E0068A406D069A404D0FB0E6816C2EC06F05C
:10189E006DA203D004EC07F0DCD068A018D069A0CC
:1018AE0016D0A5DD040E386E200E0401026F040E54
:1018BE00036F080E016F000E0015006E00C000F4DD
:1018CE008C0E0011006E00C000F4FE0E681668A8A3
:1018DE0006D069A804D0D3EC07F0EF0E681668ACFA
:1018EE0004D069AC02D0BF0E681668AA04D069AAEB
:1018FE0002D063EC07F068A202D069B26A6A040EE5
:10190E00385C03E204EC07F0A4D069A6A0D0000175
:10191E00D86B040ED85DD8B09AD068A694D06CCF90
:10192E0076F0F70E6816780E7615016E0150000AE5
:10193E00D8A488D0FD0E7615016E026AFF0E02162F
:10194E00000E021802E1000E01186DE17E0E7615F2
:10195E00016E01C003F00332039E03C000F0000EBF
:10196E00016E003600900136003600900136000EF2
:10197E000024026E040E0120036E02C06FF003C03D
:10198E0070F002C095F003C096F0040E9519006E2B
:10199E0000C095F002C0E9FF03C0EAFFEECF00F0F1
:1019AE0000C001F03C0E01160132019E0132019E73
:1019BE0001500D0A35E1020E6F25E96E000E702101
:1019CE00EA6EEECF01F0EECF02F00250040A02E111
:1019DE00280E011822E1020E6F25E16E000E702115
:1019EE00E26E200EE66E040EE66ED76B080ED75D25
:1019FE0014E2200EE16E040EE26ED751E126D8B04D
:101A0E00E22A280EE96E040EEA6ED751E926D8B006
:101A1E00EA2AEECFE6FFD72BE9D7EEEC06F002D09E
:101A2E00CAEC06F00ED0FD0E7615016E026AFF0EA0
:101A3E000216000E021802E1040E011802E181ECFA
:101A4E0007F000D001D003D00001D82B62D704ECF0
:041A5E0007F012007B
:101A620003500718D8A445EF0DF002500618D8A469
:101A720045EF0DF001500518D8A445EF0DF00050C8
:0E1A82000418D8B4D8841200D89412001200B0
:101A90000C6A0E6A0250D8A461EF0DF001C002F08A
:101AA00000C001F0006A0E860250D8A461EF0DF06C
:101AB00001C002F0016A0E960E880250D8B473EF8E
:101AC0000DF00E50035ED8A4D8A079EF0DF0D89099
:101AD00002BE7FEF0DF0003601360236032E68EFAE
:101AE0000DF079EF0DF0010E0C6E69EC01F083EF53
:101AF0000DF0020E0C6EEEEC00F083EF0DF0040E14
:081B00000C6EFBEC00F012007A
:101B08000B6A0C6A0A6A086A0350D8B40CEF0EF024
:101B1800028E9E0E035E03BE97EF0DF0D8B497EFCA
:101B28000DF0FCEF0DF0036C080E035CD8A0C9EFB4
:101B38000DF0036E083600C008F001C000F002C0C6
:101B480001F0026A080E035CD8A0C9EF0DF0036E1D
:101B5800083600C008F001C000F0016A080E035CF6
:101B6800D8A0C9EF0DF0036E083600C008F0006A6F
:101B7800080E035CD8A0C9EF0DF0036E0836086A9A
:101B88000350D8A4D890D5EF0DF00350D8B4D5EFB2
:101B98000DF0D8900232013200320832032ECDEF18
:101BA8000DF00BBC08A0E6EF0DF0D8A0E6EF0DF0A5
:101BB800082AD8B4002AD8B4012AD8B4022A02BE06
:101BC80010EF0EF00AAE0CEF0EF0021E011E001E02
:101BD800081E082AD8B4002AD8B4012AD8B4022A80
:101BE8000CEF0EF0026A016A006A086A0CEF0EF048
:101BF8000B800BAE16EF0EF0026A0AAE16EF0EF06F
:101C0800026E016E006E086E0A36023216EF0EF092
:101C1800000E0C6A17EF0EF0010E0C6E06EC07F0C2
:101C280017EF0EF0FF0E0250036E0150026E0050C7
:081C3800016E0850006E12005D
:101C40000001DA6BDB6BDC6B020ED725F66E000E43
:101C5000D821F76E000ED921F86E0900F5CF05F0F6
:101C6000030ED725F66E000ED821F76E000ED9218F
:101C7000F86E0900F5CF00F000C003F0000E046E0E
:101C800003C001F0006A05500024066E000E01201A
:101C9000076ED7C008F0D8C009F0D9C00AF0010E0D
:101CA0000824F66E000E0920F76E000E0A20F86E6A
:101CB0000900F5CF01F00150020A1BE1060E0824CD
:101CC000F66E000E0920F76E000E0A20F86E09006D
:101CD000F5CF01F00150DA5D0CE2060E0824F66E35
:101CE000000E0920F76E000E0A20F86E0900F5CFED
:101CF000DAF0010E0824F66E000E0920F76E000ED1
:101D00000A20F86E0900F5CF01F00150040A1BE12A
:101D1000080E0824F66E000E0920F76E000E0A2049
:101D2000F86E0900F5CF01F00150DA5D0CE2080E03
:101D30000824F66E000E0920F76E000E0A20F86ED9
:101D40000900F5CFDAF008C0F6FF09C0F7FF0AC0B6
:101D5000F8FF0900F5CF00F00050DB25016E000E02
:101D6000DC21026E01C0DBF002C0DCF00750025C37
:101D700002E10650015C01E30FD008C0F6FF09C084
:101D8000F7FF0AC0F8FF0900F5CF00F00050082661
:0E1D9000000E09220A2283D7DAC000F01200EA
:101D9E000450000A08E10550000A05E1FF0E006E2E
:101DAE007F0E016E58D00D6A096A086A0150001044
:101DBE00D8B4000C015005180A6E0ABE0D1E0B6A2F
:101DCE0005AE05D0041E051E042AD8B4052A01AEA0
:101DDE0005D0001E011E002AD8B4012A015005109C
:101DEE000A6E0ABE10D03CEC0AF00BB020D00DAE3D
:101DFE00000C001E011E002AD8B4012A081E091E5E
:101E0E00082AD8B4092A000C05AE0DD001BE07D0A1
:101E1E000150096E0050086E016A006AE8D7016A27
:101E2E00006A002A000C011E001E0B2ADDD7082AAC
:101E3E00D8B4092A0450085CD8A4D9D70550095C37
:101E4E00D8A4D5D7096A086A002AD8B4012A01AEE7
:081E5E00CED70000FF0C1200BA
:0A1E6600D08EA28AA08AF28E12002C
:101E7000000E006E5C0E016E000E026E0E0E00244F
:101E8000F66E000E0120F76E000E0220F86E0900BB
:101E9000F5CF03F003C004F00F0E0024F66E000E21
:101EA0000120F76E000E0220F86E0900F5CF01F058
:101EB0000150035C12E2000E006E5C0E016E000E1B
:101EC000026E0F0E0024F66E000E0120F76E000E5B
:101ED0000220F86E0900F5CF04F0000E006E5C0ED3
:101EE000016E000E026E100E0024F66E000E012030
:101EF000F76E000E0220F86E0900F5CF01F00150D8
:101F0000045C12E2000E006E5C0E016E000E026EAA
:101F1000100E0024F66E000E0120F76E000E022057
:0E1F2000F86E0900F5CF04F004C000F01200C6
:101F2E00000E0001D81902E1000ED71902E1016A74
:101F3E000AD0D7C0E9FFD8C0EAFFEECF00F0000EFE
:0C1F4E0000BE010E016E01C000F0120088
:101F5A000001D851000A12E0D7C000F0000E016E4D
:101F6A00003600900136430E0024E96E000E01206F
:101F7A00EA6EEECF04F0EECF05F011D0D7C000F034
:101F8A00000E016E003600900136830E0024E96EC1
:101F9A00000E0120EA6EEECF04F0EECF05F0020E3D
:101FAA000424E16E000E0520E26ED9C0E6FFDAC015
:101FBA00E6FF010E0424E16E000E0520E26EDBC08E
:101FCA00E6FF04C0E9FF05C0EAFFEECF00F004C057
:101FDA00E1FF05C0E2FF400E0014E66E04C0E9FF0F
:101FEA0005C0EAFFEECF00F004C0E1FF05C0E2FF42
:101FFA00880E0010E66ED851000A1BE0D7C000F028
:10200A00000E016E003600900136430E0024026E67
:10201A00000E0120036E02C0E9FF03C0EAFF040EAE
:10202A00EE18006E02C0E1FF03C0E2FF00C0E6FF47
:10203A001AD0D7C000F0000E016E003600900136AB
:10204A00830E0024026E000E0120036E02C0E9FF17
:10205A0003C0EAFF040EEE18006E02C0E1FF03C0DF
:10206A00E2FF00C0E6FF04C000F005C001F0120064
:10207A000B6A0C6A086A0350D8B4C1EF10F002C0A8
:10208A000AF0028E9E0E035E03AEB1EF10F0036CEF
:10209A00080E035CD8A07EEF10F0036E083600C06D
:1020AA0008F001C000F002C001F0026A080E035CE9
:1020BA00D8A07EEF10F0036E083600C008F001C009
:1020CA0000F0016A080E035CD8A07EEF10F0036EE0
:1020DA00083600C008F0006A080E035CD8A07EEF3C
:1020EA0010F0036E0836086A0350D8A4D8908AEF15
:1020FA0010F00350D8B48AEF10F0D89002320132AF
:10210A0000320832032E82EF10F00BBC08A09BEFBE
:10211A0010F0D8A09BEF10F0082AD8B4002AD8B43F
:10212A00012AD8B4022A02BEC5EF10F00AAEC1EFE6
:10213A0010F0021E011E001E081E082AD8B4002A2A
:10214A00D8B4012AD8B4022AC1EF10F0026A016A8F
:10215A00006A086AC1EF10F00B800BAECCEF10F0EA
:10216A00026A0AAECCEF10F0026E016E006E086EC3
:10217A000A360232CCEF10F00C6A000ECDEF10F0E6
:10218A00010E0C6E000E06EC07F0CDEF10F0FF0EFC
:10219A000250036E0150026E0050016E0850006E2C
:0221AA00120021
:1021AC000050086E0150006E0250016E0350026E1A
:1021BC00036A0B6A0C6A9E0E036E0A6A020E0C6EA0
:0621CC005FEC04F01200BC
:1021D200800E0001D719006E800E000A005CD8B094
:1021E2006DD1D7510008016E01C0D7F0800E0118E1
:1021F200006E800E6E0A005CD8A0C0D0640E046E21
:10220200D7C000F014EC07F0120E0024056E000E89
:1022120000BEFF0E066E000E062205C000F006C0CC
:1022220001F0000E06BEFF0E026E036E0036009035
:102232000136023603360036009001360236033686
:102242006A0E0024F66E5A0E0120F76E000E02206E
:10225200F86E0900F5CFD8F00900F5CFD9F00900E2
:10226200F5CFDAF00900F5CFDBF0640E046ED7C0CB
:1022720000F014EC07F008C000F00A0E046E14EC33
:1022820007F0090E0024056E000E00BEFF0E066E5A
:10229200000E062205C000F006C001F0000E06BEC8
:1022A200FF0E026E036E00360090013602360336D0
:1022B200003600900136023603366A0E0024F66EAE
:1022C2005A0E0120F76E000E0220F86E0900F5CFBB
:1022D20000F00900F5CF01F00900F5CF02F0090086
:1022E200F5CF03F0D8C004F0D9C005F0DAC006F08B
:1022F200DBC007F068EC0AF000C0D8F001C0D9F0EA
:1023020002C0DAF003C0DBF00A0E046ED7C000F0A0
:1023120014EC07F008C000F000C001F0000E00BE8F
:10232200FF0E026E036E046E013601900236033612
:102332000436013601900236033604366A0E012451
:10234200F66E5A0E0220F76E000E0320F86E090098
:10235200F5CF00F00900F5CF01F00900F5CF02F04A
:102362000900F5CF03F0D8C004F0D9C005F0DAC0F7
:1023720006F0DBC007F068EC0AF007D2800E0A0A0A
:10238200006E800ED719005C71E20A0E046ED7C08F
:1023920000F014EC07F0090E0024056E000E00BEDA
:1023A200FF0E066E000E062205C000F006C001F008
:1023B200000E06BEFF0E026E036E0036009001365E
:1023C20002360336003600900136023603366A0EB4
:1023D2000024F66E5A0E0120F76E000E0220F86EEF
:1023E2000900F5CFD8F00900F5CFD9F00900F5CFF3
:1023F200DAF00900F5CFDBF00A0E046ED7C000F068
:1024020014EC07F008C000F000C001F0000E00BE9E
:10241200FF0E026E036E046E013601900236033621
:102422000436013601900236033604366A0E012460
:10243200F66E5A0E0220F76E000E0320F86E0900A7
:10244200F5CF00F00900F5CF01F00900F5CF02F059
:102452000900F5CF03F0D8C004F0D9C005F0DAC006
:1024620006F0DBC007F068EC0AF08FD1D7C000F0AD
:10247200000ED7BFFF0E016E026E036E0036009093
:102482000136023603360036009001360236033634
:102492006A0E0024F66E5A0E0120F76E000E02201C
:1024A200F86E0900F5CF00F00900F5CF01F0090040
:1024B200F5CF02F00900F5CF03F067D1800ED719EE
:1024C200006E800E6E0A005CD8A0C0D0640E046E4E
:1024D200D7C000F014EC07F0120E0024056E000EB7
:1024E20000BEFF0E066E000E062205C000F006C0FA
:1024F20001F0000E06BEFF0E026E036E0036009063
:1025020001360236033600360090013602360336B3
:10251200360E0024F66E5A0E0120F76E000E0220CF
:10252200F86E0900F5CFD8F00900F5CFD9F009000F
:10253200F5CFDAF00900F5CFDBF0640E046ED7C0F8
:1025420000F014EC07F008C000F00A0E046E14EC60
:1025520007F0090E0024056E000E00BEFF0E066E87
:10256200000E062205C000F006C001F0000E06BEF5
:10257200FF0E026E036E00360090013602360336FD
:1025820000360090013602360336360E0024F66E0F
:102592005A0E0120F76E000E0220F86E0900F5CFE8
:1025A20000F00900F5CF01F00900F5CF02F00900B3
:1025B200F5CF03F0D8C004F0D9C005F0DAC006F0B8
:1025C200DBC007F068EC0AF000C0D8F001C0D9F017
:1025D20002C0DAF003C0DBF00A0E046ED7C000F0CE
:1025E20014EC07F008C000F000C001F0000E00BEBD
:1025F200FF0E026E036E046E013601900236033640
:10260200043601360190023603360436360E0124B2
:10261200F66E5A0E0220F76E000E0320F86E0900C5
:10262200F5CF00F00900F5CF01F00900F5CF02F077
:102632000900F5CF03F0D8C004F0D9C005F0DAC024
:1026420006F0DBC007F068EC0AF09FD0800E0A0AA1
:10265200006E800ED719005C71E20A0E046ED7C0BC
:1026620000F014EC07F0090E0024056E000E00BE07
:10267200FF0E066E000E062205C000F006C001F035
:10268200000E06BEFF0E026E036E0036009001368B
:102692000236033600360090013602360336360E15
:1026A2000024F66E5A0E0120F76E000E0220F86E1C
:1026B2000900F5CFD8F00900F5CFD9F00900F5CF20
:1026C200DAF00900F5CFDBF00A0E046ED7C000F095
:1026D20014EC07F008C000F000C001F0000E00BECC
:1026E200FF0E026E036E046E01360190023603364F
:1026F200043601360190023603360436360E0124C2
:10270200F66E5A0E0220F76E000E0320F86E0900D4
:10271200F5CF00F00900F5CF01F00900F5CF02F086
:102722000900F5CF03F0D8C004F0D9C005F0DAC033
:1027320006F0DBC007F068EC0AF027D0D7C000F043
:10274200000ED7BFFF0E016E026E036E00360090C0
:102752000136023603360036009001360236033661
:10276200360E0024F66E5A0E0120F76E000E02207D
:10277200F86E0900F5CF00F00900F5CF01F009006D
:0C278200F5CF02F00900F5CF03F01200C3
:10278E000B6A0A6A096A086A0E6A0334083604502C
:10279E00085E0550D8A0053C095E0650D8A0063C40
:1027AE000A5E0750D8A0073C0B5EE86AD8A0010E5F
:1027BE000E5E0336070E0C6E0334083609360A36E3
:1027CE000B360E36045003A012D0085E0550D8A06A
:1027DE00053C095E0650D8A0063C0A5E0750D8A0FC
:1027EE00073C0B5EE86AD8A0010E0E5E11D00826DB
:1027FE000550D8B0053C09260650D8B0063C0A262E
:10280E000750D8B0073C0B26E86AD8B0010E0E264A
:10281E0003360C2ED1D70234083609360A360B365B
:10282E000E36045003A012D0085E0550D8A0053C09
:10283E00095E0650D8A0063C0A5E0750D8A0073C99
:10284E000B5EE86AD8A0010E0E5E11D00826055068
:10285E00D8B0053C09260650D8B0063C0A260750CB
:10286E00D8B0073C0B26E86AD8B0010E0E26023609
:10287E00070E0C6E0234083609360A360B360E3643
:10288E00045002A012D0085E0550D8A0053C095E87
:10289E000650D8A0063C0A5E0750D8A0073C0B5E37
:1028AE00E86AD8A0010E0E5E11D008260550D8B0E9
:1028BE00053C09260650D8B0063C0A260750D8B06B
:1028CE00073C0B26E86AD8B0010E0E2602360C2EF7
:1028DE00D1D70134083609360A360B360E36045077
:1028EE0002A012D0085E0550D8A0053C095E065025
:1028FE00D8A0063C0A5E0750D8A0073C0B5EE86ADB
:10290E00D8A0010E0E5E11D008260550D8B0053C99
:10291E0009260650D8B0063C0A260750D8B0073C08
:10292E000B26E86AD8B0010E0E260136070E0C6E85
:10293E000134083609360A360B360E36045001A01D
:10294E0012D0085E0550D8A0053C095E0650D8A0EE
:10295E00063C0A5E0750D8A0073C0B5EE86AD8A07A
:10296E00010E0E5E11D008260550D8B0053C092682
:10297E000650D8B0063C0A260750D8B0073C0B26A6
:10298E00E86AD8B0010E0E2601360C2ED1D70034CF
:10299E00083609360A360B360E36045001A012D010
:1029AE00085E0550D8A0053C095E0650D8A0063C2E
:1029BE000A5E0750D8A0073C0B5EE86AD8A0010E4D
:1029CE000E5E11D008260550D8B0053C09260650DB
:1029DE00D8B0063C0A260750D8B0073C0B26E86A4A
:1029EE00D8B0010E0E260036070E0C6E00340836D7
:1029FE0009360A360B360E36045000A012D0085E89
:102A0E000550D8A0053C095E0650D8A0063C0A5ECB
:102A1E000750D8A0073C0B5EE86AD8A0010E0E5EE8
:102A2E0011D008260550D8B0053C09260650D8B05E
:102A3E00063C0A260750D8B0073C0B26E86AD8B0E9
:102A4E00010E0E2600360C2ED1D700B00ED004503B
:102A5E0008260550D8B0053C09260650D8B0063CCD
:0C2A6E000A260750D8B0073C0B261200C7
:102A7A006E0E0001D75DD8A0CAD0640E046ED7C00E
:102A8A0000F0D8EC07F0120E0024056E066A000E5C
:102A9A00062205C000F006C001F0000E06BEFF0EB9
:102AAA00026E036E00360090013602360336003697
:102ABA0000900136023603366A0E0024F66E5A0E6C
:102ACA000120F76E000E0220F86E0900F5CF00F023
:102ADA000900F5CF01F00900F5CF02F00900F5CFA2
:102AEA0003F0000E046E000E056E000E066E7E0EDA
:102AFA00076E68EC0AF000C0D8F001C0D9F002C035
:102B0A00DAF003C0DBF0640E046ED7C000F0D8EC34
:102B1A0007F008C000F00A0E046ED8EC07F0090EA0
:102B2A000024056E066A000E062205C000F006C0E3
:102B3A0001F0000E06BEFF0E026E036E0036009014
:102B4A000136023603360036009001360236033665
:102B5A006A0E0024F66E5A0E0120F76E000E02204D
:102B6A00F86E0900F5CF00F00900F5CF01F0090071
:102B7A00F5CF02F00900F5CF03F0D8C004F0D9C0B0
:102B8A0005F0DAC006F0DBC007F068EC0AF000C016
:102B9A00D8F001C0D9F002C0DAF003C0DBF00A0EA7
:102BAA00046ED7C000F0D8EC07F008C000F000C0EF
:102BBA0001F0000E026E036E046E013601900236B9
:102BCA0003360436013601900236033604366A0E9D
:102BDA000124F66E5A0E0220F76E000E0320F86EDC
:102BEA000900F5CF00F00900F5CF01F00900F5CF93
:102BFA0002F00900F5CF03F0D8C004F0D9C005F0FF
:102C0A00DAC006F0DBC007F068EC0AF0B1D0D751A1
:102C1A000A08D8B07ED00A0E046ED7C000F0D8ECED
:102C2A0007F0090E0024056E066A000E062205C08A
:102C3A0000F006C001F0000E06BEFF0E026E036E23
:102C4A00003600900136023603360036009001360F
:102C5A00023603366A0E0024F66E5A0E0120F76E0B
:102C6A00000E0220F86E0900F5CF00F00900F5CF3A
:102C7A0001F00900F5CF02F00900F5CF03F0000ECC
:102C8A00046E000E056E000E066E7E0E076E68EC70
:102C9A000AF000C0D8F001C0D9F002C0DAF003C0CF
:102CAA00DBF00A0E046ED7C000F0D8EC07F008C0BB
:102CBA0000F000C001F0000E026E036E046E0136D1
:102CCA000190023603360436013601900236033685
:102CDA0004366A0E0124F66E5A0E0220F76E000EB2
:102CEA000320F86E0900F5CF00F00900F5CF01F0D6
:102CFA000900F5CF02F00900F5CF03F0D8C004F0BF
:102D0A00D9C005F0DAC006F0DBC007F068EC0AF0BB
:102D1A002FD0D7C000F0000E016E026E036E00368F
:102D2A00009001360236033600360090013602362C
:102D3A0003366A0E0024F66E5A0E0120F76E000E54
:102D4A000220F86E0900F5CF00F00900F5CF01F076
:102D5A000900F5CF02F00900F5CF03F0000E046E6A
:102D6A00000E056E000E066E7E0E076E68EC0AF007
:022D7A00120045
:102D7C0000C008F00150006E016A026A036A0B6A17
:102D8C000C6A016A026A036A960E036E0A6A00AE46
:102D9C00D6EF16F0081E001E082AD8B4002A0A8E98
:102DAC0000C001F008C000F0086A026A48EC0DF09F
:022DBC00120003
:102DBE003850000A0CE16D6A696ABBEC06F033EC20
:102DCE000FF06DB602D06D86FCD7010E386E120074
:102DDE00200E385C03E36DB201D002D0006A4AD0F7
:102DEE007BC0D7F07CC0D8F097EC0FF0005241E1D9
:102DFE00B2C0D7F0010ED86FAFC0D9F0B0C0DAF0C4
:102E0E00B1C0DBF0ADEC0FF000C07BF001C07CF088
:102E1E00776B786B796B7A6B7BC0D7F07CC0D8F010
:102E2E0097EC0FF0005210E0010E016E0150000AF7
:102E3E0002E12FEC0CF000017751781179117A1123
:102E4E0002E0006A17D0E8D77BC0B3F07CC0B4F0C4
:102E5E00000E7C1902E1000E7B1909E0010EB3256C
:102E6E00E96E000EB421EA6EEECF00F003D0006AD8
:062E7E0001D0006A120001
:102E84000001CF6BD06BC36BC46BB1C000F0B2C098
:102E940001F0B3C002F0010EB127000EB223B32338
:102EA40000C0F6FF01C0F7FF02C0F8FF0900F5CF2C
:102EB40000F000C0C0F00052D8B452EF27F0C05167
:102EC400250A0BE0AFC0E1FFB0C0E2FFC0C0E6FFDF
:102ED400AF4BB02BCF4BD02BD8D7C16BC26BC36BCE
:102EE400C46B23D0C387010EB127000EB223B323D2
:102EF40059D0C381010EB127000EB223B32352D09F
:102F0400C383010EB127000EB223B3234BD0C48771
:102F1400010EB127000EB223B32344D0C385010EA2
:102F2400B127000EB223B3233DD0B1C0F6FFB2C027
:102F3400F7FFB3C0F8FF0900F5CF01F001502D0AE7
:102F4400D1E0B1C0F6FFB2C0F7FFB3C0F8FF09008B
:102F5400F5CF01F00150200ACCE0B1C0F6FFB2C0B9
:102F6400F7FFB3C0F8FF0900F5CF01F001502B0AB9
:102F7400C7E0B1C0F6FFB2C0F7FFB3C0F8FF090065
:102F8400F5CF01F00150230AC2E0B1C0F6FFB2C090
:102F9400F7FFB3C0F8FF0900F5CF01F00150300A84
:102FA400BDE001D09ED7C3A301D0C391C3A701D074
:102FB400C395B1C0F6FFB2C0F7FFB3C0F8FF090074
:102FC400F5CF00F0000E016E00C0D7F0FEEC0AF061
:102FD400005236E0C16BC26BC1C000F0C2C001F048
:102FE4000A0E046E000E056E57EC00F0B1C0F6FF39
:102FF400B2C0F7FFB3C0F8FF0900F5CF02F00250EA
:103004000024C16F000E0120C26F300EC15F000E9C
:10301400C25B010EB127000EB223B323B1C0F6FF89
:10302400B2C0F7FFB3C0F8FF0900F5CF00F0000EFF
:10303400016E00C0D7F0FEEC0AF00052CDE133D0AF
:10304400B1C0F6FFB2C0F7FFB3C0F8FF0900F5CF77
:1030540001F001502A0A27E1B4C0E9FFB5C0EAFF34
:10306400EECF00F0EECF01F000C0E9FF01C0EAFFAF
:10307400EECFC1F0EECFC2F0B4C0E9FFB5C0EAFFB5
:10308400020EEE24006E000EEE20016EB4C0E1FFCD
:10309400B5C0E2FF00C0E6FF01C0E6FF010EB127A4
:1030A400000EB223B323B1C0F6FFB2C0F7FFB3C022
:1030B400F8FF0900F5CF01F001502E0A70E1010E6E
:1030C400B127000EB223B323B1C0F6FFB2C0F7FF9D
:1030D400B3C0F8FF0900F5CF01F001502A0A28E136
:1030E400B4C0E9FFB5C0EAFFEECF00F0EECF01F0C7
:1030F40000C0E9FF01C0EAFFEECFBEF0EECFBFF0A3
:10310400B4C0E9FFB5C0EAFF020EEE24006E000E63
:10311400EE20016EB4C0E1FFB5C0E2FF00C0E6FFDF
:1031240001C0E6FF010EB127000EB223B32336D04F
:10313400BE6BBF6BB1C0F6FFB2C0F7FFB3C0F8FF00
:103144000900F5CF00F0000E016E00C0D7F0FEECD0
:103154000AF0005223E0BEC000F0BFC001F00A0E26
:10316400046E000E056E57EC00F0B1C0F6FFB2C05D
:10317400F7FFB3C0F8FF0900F5CF02F002500024B6
:10318400BE6F000E0120BF6F300EBE5F000EBF5B2E
:10319400010EB127000EB223B323CCD703D0BE6BEC
:1031A400BF6BC489B1C000F0B2C001F0B3C002F07B
:1031B400010EB127000EB223B32300C0F6FF01C0F5
:1031C400F7FF02C0F8FF0900F5CFC0F0F9D0CFC077
:1031D40000F0D0C001F056EF27F0C389E3D7C485CF
:1031E4002ED1C38BC4812BD1C48329D1C38D27D1C4
:1031F40026D1C38BC38F23D1B4C0E9FFB5C0EAFF86
:10320400EECF00F0EECF01F000C0E9FF01C0EAFF0D
:10321400EECFCBF0EECFCCF0B4C0E9FFB5C0EAFFFF
:10322400020EEE24006E000EEE20016EB4C0E1FF2B
:10323400B5C0E2FF00C0E6FF01C0E6FF000ECC19F6
:1032440002E1000ECB1904E1290ECB6F000ECC6F06
:10325400CD6BCE6BCD51CB25E96ECE51CC21EA6E30
:10326400EE520BE0010ECD25006E000ECE21016E54
:1032740000C0CDF001C0CEF0EDD7BE51BF110AE0C1
:10328400CE51BF5D02E1CD51BE5D04E2BEC0CDF0C2
:10329400BFC0CEF0C251CE5D02E1C151CD5D05E2A9
:1032A400CD51C15FCE51C25B02D0C16BC26BC3B7FB
:1032B40016D0C1C000F0C2C001F0010EC15F000E03
:1032C400C25B005001100BE0AFC0E1FFB0C0E2FFF1
:1032D400200EE66EAF4BB02BCF4BD02BEAD7CDC030
:1032E40002F0CEC003F0010ECD5D006E000ECE598B
:1032F400016E00C0CDF001C0CEF00250031019E001
:10330400CBC0E9FFCCC0EAFFAFC0E1FFB0C0E2FF31
:10331400EECFE6FFAF4BB02B010ECB25006E000EB7
:10332400CC21016E00C0CBF001C0CCF0CF4BD02B30
:10333400D6D7C3A716D0C1C000F0C2C001F0010E99
:10334400C15F000EC25B005001100BE0AFC0E1FF93
:10335400B0C0E2FF200EE66EAF4BB02BCF4BD02BAC
:10336400EAD793D5B4C0E9FFB5C0EAFFEECF00F0C9
:10337400EECF01F000C0E9FF01C0EAFFEECFC0F0DC
:10338400B4C0E9FFB5C0EAFF020EEE24006E000EE1
:10339400EE20016EB4C0E1FFB5C0E2FF00C0E6FF5D
:1033A40001C0E6FFC00ECB6F000ECC6F010ECD6FD7
:1033B400000ECE6F62D7C00EC313000EC4133FD0ED
:1033C400C051000AD8B403D7C0516C0AD8B405D789
:1033D400C0514C0AD8B401D7C051660AD8B4FFD63C
:1033E400C051450AD8B4FDD6C051650AD8B4FAD63E
:1033F400C051670AD8B4F8D6C0516F0AD8B4F6D60B
:10340400C051640AD8B4F4D6C051690AD8B4F0D60D
:10341400C051700AD8B4EDD6C051580AD8B4E9D610
:10342400C051780AD8B4E6D6C051730AD8B4E4D6E9
:10343400C051630A97E0C051750ABDE0B3D7000ECE
:10344400C315006EC451070B016E00500110D8B4AF
:10345400F9EF22F0C4A904D0060EBE6F000EBF6FB0
:10346400B4C0E9FFB5C0EAFFEECF00F0EECF01F043
:1034740000C0E9FF01C0EAFFEECFC5F0EECFC6F011
:10348400EECFC7F0EECFC8F0B4C0E9FFB5C0EAFF95
:10349400040EEE24006E000EEE20016EB4C0E1FFB7
:1034A400B5C0E2FF00C0E6FF01C0E6FF046A056A9A
:1034B400066A076AC5C000F0C6C001F0C7C002F0C2
:1034C400C8C003F00AEC0BF0010ED8B0000E006E79
:1034D400005205E0C77F030EC313000EC413C96B6B
:1034E400CA6BC5C000F0C6C001F0C7C002F0C8C0B6
:1034F40003F0046A056A066A076A31EC0DF0000EEF
:10350400D8A4010E006E0052D8B48AD0C8C000F00E
:10351400016A026A036AFF0E0016000E01167E0E8F
:10352400005E000E015A00C0C9F001C0CAF0010ECD
:10353400005E000E015A00C0C9F001C0CAF0030EBB
:10354400046E000E056E57EC00F000C0C9F001C017
:10355400CAF00A0E046E000E056ECFEC0EF000C029
:10356400C9F001C0CAF0800E0118026E800E025C20
:1035740002E1000E005C05E2010E0001C95F000ECD
:10358400CA5B0001C9510008D76FE9EC10F0C5C04F
:1035940004F0C6C005F0C7C006F0C8C007F068EC68
:1035A4000AF000C0CBF001C0CCF002C0CDF003C0E3
:1035B400CEF0000E046E000E056E000E066E7F0E39
:1035C400076ECBC000F0CCC001F0CDC002F0CEC07D
:1035D40003F00AEC0BF0010ED8B0000E006E00529E
:1035E40005E0010EC95F000ECA5B1AD0000E046E1E
:1035F400000E056E200E066E820E076ECBC000F024
:10360400CCC001F0CDC002F0CEC003F00AEC0BF048
:10361400000ED8B0010E006E005202E0C94BCA2B56
:10362400800E006E800ECA19005C02E1C9510008C8
:1036340003E3010EC06F02D0C9C0C0F0C4B118D0FA
:10364400C4A315D0800ECA19006E7F0E005C02E17F
:10365400FC0EC95D0BE3800ECA19006E800EBF1903
:10366400005C02E1BE51C95D01E201D001D0F1D399
:10367400BE51BF1106E0C4A304D0010EBE5F000E0C
:10368400BF5B000E006EBF51005C02E1BE51080832
:1036940003E2080EC06F02D0BEC0C0F0C5C000F087
:1036A400C6C001F0C7C002F0C8C003F0046A056ACE
:1036B400066A076A31EC0DF0000ED8A4010E006E04
:1036C4000052D8B44BD1C9C0D7F0E9EC10F000C017
:1036D40004F001C005F002C006F003C007F0C5C045
:1036E40000F0C6C001F0C7C002F0C8C003F071EC1E
:1036F4000BF000C0C5F001C0C6F002C0C7F003C0A3
:10370400C8F00001C0510008D76FE9EC10F000C008
:1037140004F001C005F002C006F003C007F0C5C004
:1037240000F0C6C001F0C7C002F0C8C003F071ECDD
:103734000BF000C0D1F001C0D2F002C0D3F003C03E
:10374400D4F0D1C0C5F0D2C0C6F0D3C0C7F0D4C045
:10375400C8F0D1C000F0D2C001F0D3C002F0D4C090
:1037640003F084EC0DF0D6EC10F000C004F001C0BE
:1037740005F002C006F003C007F0D1C000F0D2C0CB
:1037840001F0D3C002F0D4C003F0FBEC0AF0000E49
:10379400046E000E056E000E066E7E0E076E0AECB9
:1037A4000BF0000ED8B0010E006E00521AE0C5C036
:1037B40000F0C6C001F0C7C002F0C8C003F0000E9C
:1037C400046E000E056E000E066E7E0E076EEBECA8
:1037D40007F000C0C5F001C0C6F002C0C7F003C0C6
:1037E400C8F0C5C000F0C6C001F0C7C002F0C8C030
:1037F40003F084EC0DF00001C051010F096E0A6A58
:10380400000E0A2209C004F00AC005F0000E0ABE28
:10381400FF0E066E076E043604900536063607362C
:1038240004360490053606360736270E0424F66E51
:103834005B0E0520F76E000E0620F86E0900F5CF2A
:1038440005F00900F5CF06F00900F5CF07F00900EF
:10385400F5CF08F00850035C08E10750025C05E16D
:103864000650015C02E10550005C1EE30001C5C086
:1038740000F0C6C001F0C7C002F0C8C003F0CD0E0E
:10388400046ECC0E056E4C0E066E7B0E076E68EC55
:103894000AF000C0C5F001C0C6F002C0C7F003C002
:1038A400C8F0C94BCA2B5AD0C5C000F0C6C001F03D
:1038B400C7C002F0C8C003F084EC0DF0C0C004F02F
:1038C400000E056E066E076E043604900536063645
:1038D400073604360490053606360736270E0424C8
:1038E400F66E5B0E0520F76E000E0620F86E0900DA
:1038F400F5CF05F00900F5CF06F00900F5CF07F084
:103904000900F5CF08F00850035C08E10750025C99
:1039140005E10650015C02E10550005C1FE2000174
:10392400C5C000F0C6C001F0C7C002F0C8C003F0B3
:10393400000E046E000E056E200E066E820E076EDB
:1039440068EC0AF000C0C5F001C0C6F002C0C7F0C0
:1039540003C0C8F0010EC95F000ECA5B0001C4A316
:1039640093D0C4B791D0800E000A006E800EBF19A8
:10397400005C02E1BE510A0804E20A0EBE6F000EAA
:10398400BF6FC5C000F0C6C001F0C7C002F0C8C018
:1039940003F084EC0DF000C0CBF001C0CCF002C009
:1039A400CDF003C0CEF0CB51CC11CD11CE1142E0FD
:1039B4000A0E046E000E056E066E076ECBC000F094
:1039C400CCC001F0CDC002F0CEC003F0C7EC13F0C0
:1039D40008C000F009C001F00AC002F00BC003F0F7
:1039E400000E046E031808E10450021805E10450A7
:1039F400011802E10050000A1DE1010EBE5F000E35
:103A0400BF5B0A0E046E000E056E066E076ECBC019
:103A140000F0CCC001F0CDC002F0CEC003F0C7EC82
:103A240013F000C0CBF001C0CCF002C0CDF003C055
:103A3400CEF0B9D7800EBF19006E800E005C02E193
:103A4400C051BE5D21E2BE51C05DD76FE9EC10F0FC
:103A540000C004F001C005F002C006F003C007F086
:103A6400C5C000F0C6C001F0C7C002F0C8C003F072
:103A740071EC0BF000C0C5F001C0C6F002C0C7F085
:103A840003C0C8F0BEC0C0F0050E0001BE25006E24
:103A9400000EBF21016E0050C15F0150C25BBE51D8
:103AA400BF1103E1C4B701D004D0010EC15F000E01
:103AB400C25B030EC315006EC4C001F0000E0116F4
:103AC4000050011004E0010EC15F000EC25BC3A5EB
:103AD40039D0C3A312D0C3A103D02D0EB66F02D028
:103AE4002B0EB66FAFC0E1FFB0C0E2FFB6C0E6FF79
:103AF400AF4BB02BCF4BD02B0CD0C3A10AD0AFC04F
:103B0400E1FFB0C0E2FF200EE66EAF4BB02BCF4B0F
:103B1400D02B800E006E800EC219005C02E1C151F0
:103B240000080FE2AFC0E1FFB0C0E2FF300EE66E66
:103B3400AF4BB02BCF4BD02B010EC15F000EC25B3D
:103B4400E8D73AD0C3B718D0800E006E800EC219E1
:103B5400005C02E1C15100080FE2AFC0E1FFB0C058
:103B6400E2FF200EE66EAF4BB02BCF4BD02B010EF5
:103B7400C15F000EC25BE8D7C3A312D0C3A103D0B8
:103B84002D0EB76F02D02B0EB76FAFC0E1FFB0C0E0
:103B9400E2FFB7C0E6FFAF4BB02BCF4BD02B0CD01E
:103BA400C3A10AD0AFC0E1FFB0C0E2FF200EE66EB1
:103BB400AF4BB02BCF4BD02BC5C000F0C6C001F02B
:103BC400C7C002F0C8C003F084EC0DF000C0CBF015
:103BD40001C0CCF002C0CDF003C0CEF0C0C000F0F4
:103BE400000E016E026E036E00360090013602363E
:103BF400033600360090013602360336270E0024C1
:103C0400F66E5B0E0120F76E000E0220F86E0900BE
:103C1400F5CF04F00900F5CF05F00900F5CF06F063
:103C24000900F5CF07F0CBC000F0CCC001F0CDC047
:103C340002F0CEC003F0C7EC13F0300E0026AFC084
:103C4400E1FFB0C0E2FF00C0E6FFAF4BB02BCF4BAB
:103C5400D02BBE51BF1103E1C4B701D06FD0AFC0A8
:103C6400E1FFB0C0E2FF2E0EE66EAF4BB02BCF4BA0
:103C7400D02BC051BE5F000EBF5BC0534DE0C007E8
:103C8400C0C000F0000E016E026E036E003600909C
:103C9400013602360336003600900136023603360A
:103CA400270E0024F66E5B0E0120F76E000E022034
:103CB400F86E0900F5CF04F00900F5CF05F009000E
:103CC400F5CF06F00900F5CF07F0CBC000F0CCC06B
:103CD40001F0CDC002F0CEC003F0C7EC13F00A0E21
:103CE400046E000E056E066E076EC7EC13F008C076
:103CF40000F009C001F00AC002F00BC003F0300E5E
:103D04000026AFC0E1FFB0C0E2FF00C0E6FFAF4B4A
:103D1400B02BCF4BD02BB1D7BE51BF110FE0AFC0EA
:103D2400E1FFB0C0E2FF300EE66EAF4BB02BCF4BDD
:103D3400D02B010EBE5F000EBF5BEED7C3AB0BD022
:103D4400AFC0E1FFB0C0E2FF450EE66EAF4BB02B53
:103D5400CF4BD02B0AD0AFC0E1FFB0C0E2FF650E5D
:103D6400E66EAF4BB02BCF4BD02B800ECA19006E32
:103D7400800E005C02E1000EC95D11E2C951000829
:103D8400C96FCA51000ECA57AFC0E1FFB0C0E2FF0D
:103D94002D0EE66EAF4BB02BCF4BD02B0AD0AFC05D
:103DA400E1FFB0C0E2FF2B0EE66EAF4BB02BCF4B62
:103DB400D02B0A0E046E000E056EC9C000F0CAC0F6
:103DC40001F0CFEC0EF0300E0026AFC0E1FFB0C022
:103DD400E2FF00C0E6FF0001AF4BB02BCF4BD02B6E
:103DE4000A0E046E000E056EC9C000F0CAC001F0D0
:103DF400CFEC0EF008C000F009C001F0300E002630
:103E0400AFC0E1FFB0C0E2FF00C0E6FF0001AF4B6E
:103E1400B02BCF4BD02BC3A71AD0800E006E800ED0
:103E2400C219005C02E1C151000811E2AFC0E1FF18
:103E3400B0C0E2FF200EE66EAF4BB02BCF4BD02BC1
:103E4400010EC15F000EC25BC151C211EFE147EF29
:103E540017F0C4A3F3D0800ECA19006E800E005C64
:103E640002E1000EC95D0AE2010EC95D006E000E9A
:103E7400CA59016E0050BE5F0150BF5BC5C000F05F
:103E8400C6C001F0C7C002F0C8C003F084EC0DF056
:103E940000C0CBF001C0CCF002C0CDF003C0CEF026
:103EA400010EC06FC0510A0A34E0C0C000F0000E19
:103EB400016E026E036E0036009001360236033640
:103EC40000360090013602360336270E0024F66EC3
:103ED4005B0E0120F76E000E0220F86E0900F5CF8C
:103EE40001F00900F5CF02F00900F5CF03F0090055
:103EF400F5CF04F00450CE5D08E10350CD5D05E13B
:103F04000250CC5D02E10150CB5D01E202D0C02B36
:103F1400C9D7C051BE5DD56F000EBF59D66FD5C08D
:103F2400BEF0D6C0BFF0CBC000F0CCC001F0CDC015
:103F340002F0CEC003F0D6EC10F000C004F001C0D3
:103F440005F002C006F003C007F0C5C000F0C6C00B
:103F540001F0C7C002F0C8C003F0FBEC0AF000C0D7
:103F6400D1F001C0D2F002C0D3F003C0D4F0D5C068
:103F7400D7F0E9EC10F0D1C004F0D2C005F0D3C002
:103F840006F0D4C007F068EC0AF0000E046E000ED0
:103F9400056E000E066E7E0E076EEBEC07F084ECE9
:103FA4000DF000C0CBF001C0CCF002C0CDF003C0D6
:103FB400CEF0BE51BF1142E00A0E046E000E056E33
:103FC400066E076ECBC000F0CCC001F0CDC002F08D
:103FD400CEC003F0C7EC13F008C000F009C001F034
:103FE4000AC002F00BC003F0000E046E031808E1CF
:103FF4000450021805E10450011802E10050000ABF
:104004001DE10A0E046E000E056E066E076ECBC02F
:1040140000F0CCC001F0CDC002F0CEC003F0C7EC7C
:1040240013F000C0CBF001C0CCF002C0CDF003C04F
:10403400CEF0010EBE5F000EBF5BBBD7800E006EDC
:10404400800EBF19005C02E1BE510C0816E3BEC02D
:10405400D7F03DEC15F0C5C004F0C6C005F0C7C0EC
:1040640006F0C8C007F0EBEC07F000C0C5F001C0D3
:10407400C6F002C0C7F003C0C8F0C5C000F0C6C097
:1040840001F0C7C002F0C8C003F0046A056A066AFA
:10409400076A31EC0DF0000ED8A4010E006E005238
:1040A400D8B477D0C5C000F0C6C001F0C7C002F0D4
:1040B400C8C003F084EC0DF0000E046E031808E190
:1040C4000450021805E10450011802E10050000AEE
:1040D40060E1800E006E800ECA19005C02E1C951D5
:1040E400010857E2C9C0D7F0E9EC10F000C004F0B1
:1040F40001C005F002C006F003C007F0C5C000F01F
:10410400C6C001F0C7C002F0C8C003F071EC0BF0E8
:104114005F0E046E700E056E090E066E810E076E3C
:104124000AEC0BF0010ED8B0000E006E005206E04F
:10413400090E0001C95F000ECA5B05D00001080E1C
:10414400C95F000ECA5BC9C0D7F0E9EC10F000C02B
:1041540004F001C005F002C006F003C007F0C5C0BA
:1041640000F0C6C001F0C7C002F0C8C003F071EC93
:104174000BF084EC0DF000C0CBF001C0CCF002C019
:10418400CDF003C0CEF00001C56BC66BC76BC86B26
:1041940038D0C5C000F0C6C001F0C7C002F0C8C026
:1041A40003F084EC0DF000C0CBF001C0CCF002C0F1
:1041B400CDF003C0CEF0CBC000F0CCC001F0CDC038
:1041C40002F0CEC003F0D6EC10F000C004F001C041
:1041D40005F002C006F003C007F0C5C000F0C6C079
:1041E40001F0C7C002F0C8C003F0FBEC0AF000C045
:1041F400C5F001C0C6F002C0C7F003C0C8F0C96B67
:10420400CA6B010EC06FC0510A0A34E0C0C000F08E
:10421400000E016E026E036E003600900136023607
:10422400033600360090013602360336270E00248A
:10423400F66E5B0E0120F76E000E0220F86E090088
:10424400F5CF01F00900F5CF02F00900F5CF03F036
:104254000900F5CF04F00450CE5D08E10350CD5DB4
:1042640005E10250CC5D02E10150CB5D01E202D0D8
:10427400C02BC9D7C051BE25006E000EBF21016EF0
:10428400C9510026CA5101220050C15F0150C25BCE
:10429400C4B704D0BE51BF1101E104D0010EC15F07
:1042A400000EC25B030EC315006EC4C001F0000E05
:1042B40001160050011004E0010EC15F000EC25B44
:1042C400C3A539D0C3A312D0C3A103D02D0EB86F98
:1042D40002D02B0EB86FAFC0E1FFB0C0E2FFB8C090
:1042E400E6FFAF4BB02BCF4BD02B0CD0C3A10AD0E1
:1042F400AFC0E1FFB0C0E2FF200EE66EAF4BB02BC3
:10430400CF4BD02B800E006E800EC219005C02E1F0
:10431400C15100080FE2AFC0E1FFB0C0E2FF300EB0
:10432400E66EAF4BB02BCF4BD02B010EC15F000E0E
:10433400C25BE8D73AD0C3B718D0800E006E800EA7
:10434400C219005C02E1C15100080FE2AFC0E1FFF5
:10435400B0C0E2FF200EE66EAF4BB02BCF4BD02B9C
:10436400010EC15F000EC25BE8D7C3A312D0C3A184
:1043740003D02D0EB96F02D02B0EB96FAFC0E1FF81
:10438400B0C0E2FFB9C0E6FFAF4BB02BCF4BD02B90
:104394000CD0C3A10AD0AFC0E1FFB0C0E2FF200E31
:1043A400E66EAF4BB02BCF4BD02BC0C000F0C00794
:1043B40000524CE0C0C000F0000E016E026E036EAD
:1043C400003600900136023603360036009001367E
:1043D40002360336270E0024F66E5B0E0120F76EBC
:1043E400000E0220F86E0900F5CF04F00900F5CFA5
:1043F40005F00900F5CF06F00900F5CF07F0CBC0B2
:1044040000F0CCC001F0CDC002F0CEC003F0C7EC88
:1044140013F00A0E046E000E056E066E076EC7ECEE
:1044240013F008C000F009C001F00AC002F00BC08C
:1044340003F0300E0026AFC0E1FFB0C0E2FF00C0C1
:10444400E6FFAF4BB02BCF4BD02BAFD7800E006E17
:10445400800ECA19005C02E1C95100080FE2AFC026
:10446400E1FFB0C0E2FF300EE66EAF4BB02BCF4B96
:10447400D02B010EC95F000ECA5BE8D7800E000A7C
:10448400006E800EBF19005C02E1BE51080803E211
:10449400080EC06F02D0BEC0C0F0C051BE5F000E97
:1044A400BF5BC05303E1C4B701D00AD0AFC0E1FF82
:1044B400B0C0E2FF2E0EE66EAF4BB02BCF4BD02B2D
:1044C400C0C0D7F0E9EC10F0C5C004F0C6C005F0D8
:1044D400C7C006F0C8C007F068EC0AF03DEC10F065
:1044E40000C0CBF001C0CCF002C0CDF003C0CEF0D0
:1044F400C0534DE0C007C0C000F0000E016E026E54
:10450400036E003600900136023603360036009002
:10451400013602360336270E0024F66E5B0E0120A8
:10452400F76E000E0220F86E0900F5CF04F00900C2
:10453400F5CF05F00900F5CF06F00900F5CF07F037
:10454400CBC000F0CCC001F0CDC002F0CEC003F06F
:10455400C7EC13F00A0E046E000E056E066E076EAD
:10456400C7EC13F008C000F009C001F00AC002F063
:104574000BC003F0300E0026AFC0E1FFB0C0E2FF75
:1045840000C0E6FFAF4BB02BCF4BD02BB1D7BE5101
:10459400BF110FE0AFC0E1FFB0C0E2FF300EE66E26
:1045A400AF4BB02BCF4BD02B010EBE5F000EBF5BC9
:1045B400EED7C3A71AD0800E006E800EC219005C1D
:1045C40002E1C151000811E2AFC0E1FFB0C0E2FF57
:1045D400200EE66EAF4BB02BCF4BD02B010EC15F3C
:1045E400000EC25BC151C211EFE147EF17F0C00EDC
:1045F400C315016EC4C002F0000E0216000E0218AC
:1046040002E1000E0118D8A480D0C3A927D0B4C0F9
:10461400E9FFB5C0EAFFEECF00F0EECF01F000C035
:10462400E9FF01C0EAFFEECFCBF0EECFCCF0EECF46
:10463400CDF0EECFCEF0B4C0E9FFB5C0EAFF040E72
:10464400EE24006E000EEE20016EB4C0E1FFB5C092
:10465400E2FF00C0E6FF01C0E6FF2FD0B4C0E9FFCF
:10466400B5C0EAFFEECF00F0EECF01F000C0E9FFE5
:1046740001C0EAFFEECF00F0EECF01F0000E01BE64
:10468400FF0E026E036E00C0CBF001C0CCF002C07E
:10469400CDF003C0CEF0B4C0E9FFB5C0EAFF020E0E
:1046A400EE24006E000EEE20016EB4C0E1FFB5C032
:1046B400E2FF00C0E6FF01C0E6FF800ECE19006EE7
:1046C400800E005C08E1000ECD5D05E1000ECC5DBE
:1046D40002E1000ECB5D18E2030EC313000EC413F7
:1046E400006A016A026A036ACB51005ECC51015A26
:1046F400CD51025ACE51035A00C0CBF001C0CCF0C8
:1047040002C0CDF003C0CEF04ED0C3A927D0B4C0B0
:10471400E9FFB5C0EAFFEECF00F0EECF01F000C034
:10472400E9FF01C0EAFFEECFCBF0EECFCCF0EECF45
:10473400CDF0EECFCEF0B4C0E9FFB5C0EAFF040E71
:10474400EE24006E000EEE20016EB4C0E1FFB5C091
:10475400E2FF00C0E6FF01C0E6FF25D0B4C0E9FFD8
:10476400B5C0EAFFEECF00F0EECF01F000C0E9FFE4
:1047740001C0EAFFEECFCBF0EECFCCF0000ECD6F50
:10478400CE6FB4C0E9FFB5C0EAFF020EEE24006E9E
:10479400000EEE20016EB4C0E1FFB5C0E2FF00C020
:1047A400E6FF01C0E6FF000EBF1902E1000EBE19CC
:1047B4000FE1000E006ECE1908E10050CD1905E19D
:1047C4000050CC1902E1CB51000A02E1BE4BBF2BD1
:1047D400C00EC315006E00C005F0AED0010EC06F50
:1047E400C0510A0A34E0C0C000F0000E016E026E2F
:1047F400036E003600900136023603360036009010
:10480400013602360336270E0024F66E5B0E0120B5
:10481400F76E000E0220F86E0900F5CF01F00900D2
:10482400F5CF02F00900F5CF03F00900F5CF04F04D
:104834000450CE5D08E10350CD5D05E10250CC5D2E
:1048440002E10150CB5D01E202D0C02BC9D782D076
:10485400010EC06FC051080A34E0C0C000F0000E61
:10486400016E026E036E0036009001360236033686
:1048740000360090013602360336B60E0024F66E7A
:104884005B0E0120F76E000E0220F86E0900F5CFD2
:1048940001F00900F5CF02F00900F5CF03F009009B
:1048A400F5CF04F00450CE5D08E10350CD5D05E181
:1048B4000250CC5D02E10150CB5D01E202D0C02B7D
:1048C400C9D748D0010EC06FC0510C0A34E0C0C033
:1048D40000F0000E016E026E036E00360090013689
:1048E4000236033600360090013602360336CE0E09
:1048F4000024F66E5A0E0120F76E000E0220F86EA8
:104904000900F5CF01F00900F5CF02F00900F5CF59
:1049140003F00900F5CF04F00450CE5D08E1035024
:10492400CD5D05E10250CC5D02E10150CB5D01E2B9
:1049340002D0C02BC9D70ED00550000AD8B44ED728
:104944000550C00AD8B44AD70550800A81E0055002
:10495400400AB8E0800E006E800EBF19005C02E1D0
:10496400BE51C05D03E2BEC0C0F00DD0800EBF19C1
:10497400006E800E005C02E1C051BE5D04E2C0C066
:10498400BEF0000EBF6FC151C2110EE0030EC3157D
:10499400006EC4C001F0000E01160050011004E0C6
:1049A400010EC15F000EC25B800EBF19006E800E47
:1049B400C219005C02E1C151BE5D05E2BE51C15F96
:1049C400BF51C25B02D0C16BC26BC40EC315016E72
:1049D400C451080B026E0250080A02E1400E01188D
:1049E40008E1C151C21104E0010EC15F000EC25BB7
:1049F4001CD0C00EC315016EC451080B026E0250C8
:104A0400080A02E1800E011810E1800E006E800E8B
:104A1400C219005C02E1C151020805E2020EC15F45
:104A2400000EC25B02D0C16BC26BC3A55DD0C3A331
:104A340012D0C3A103D02D0EBA6F02D02B0EBA6FC1
:104A4400AFC0E1FFB0C0E2FFBAC0E6FFAF4BB02B8E
:104A5400CF4BD02B34D0C3A10BD0AFC0E1FFB0C03B
:104A6400E2FF200EE66EAF4BB02BCF4BD02B27D0FE
:104A7400C00EC315016EC451080B026E0250080A21
:104A840002E1800E01181BE1AFC0E1FFB0C0E2FFFC
:104A9400300EE66EAF4BB02BCF4BD02BC3AB03D055
:104AA400580EBB6F02D0780EBB6FAFC0E1FFB0C031
:104AB400E2FFBBC0E6FFAF4BB02BCF4BD02BC151B5
:104AC400C21111E0AFC0E1FFB0C0E2FF300EE66EEC
:104AD400AF4BB02BCF4BD02B010EC15F000EC25B8E
:104AE400C151C211EFE174D0C151C21113E0C3B777
:104AF40011D0AFC0E1FFB0C0E2FF200EE66EAF4BB5
:104B0400B02BCF4BD02B010EC15F000EC25BC15145
:104B1400C211EFE1C3A312D0C3A103D02D0EBC6F09
:104B240002D02B0EBC6FAFC0E1FFB0C0E2FFBCC02F
:104B3400E6FFAF4BB02BCF4BD02B0CD0C3A10AD088
:104B4400AFC0E1FFB0C0E2FF200EE66EAF4BB02B6A
:104B5400CF4BD02BC00EC315016EC451080B026E8F
:104B64000250080A02E1400E01180BE1AFC0E1FF58
:104B7400B0C0E2FF300EE66EAF4BB02BCF4BD02B64
:104B840027D0C00EC315016EC451080B026E02502B
:104B9400080A02E1800E01181BE1AFC0E1FFB0C0BA
:104BA400E2FF300EE66EAF4BB02BCF4BD02BC3AB36
:104BB40003D0580EBD6F02D0780EBD6FAFC0E1FFB9
:104BC400B0C0E2FFBDC0E6FFAF4BB02BCF4BD02B44
:104BD400800E006E800EBF19005C02E1BE51C05D04
:104BE4000BE2AFC0E1FFB0C0E2FF300EE66EAF4BA8
:104BF400B02BCF4BD02BECD7BEC000F0BFC001F020
:104C0400010EBE5F000EBF5B00500110D8B42AD164
:104C1400C00EC315006E00C0D1F00AD1BEC000F0B2
:104C2400BFC001F0000EBFBFFF0E026E036E003660
:104C34000090013602360336003600900136023603
:104C44000336270E0024F66E5B0E0120F76E000E6D
:104C54000220F86E0900F5CF04F00900F5CF05F045
:104C64000900F5CF06F00900F5CF07F0CBC000F03E
:104C7400CCC001F0CDC002F0CEC003F0C7EC13F0FD
:104C84000A0E046E000E056E066E076EC7EC13F076
:104C940008C000F009C001F00AC002F00BC003F024
:104CA400300E0024C06FD3D0C3AB45D0BEC000F0DB
:104CB400BFC001F0000EBFBFFF0E026E036E0036D0
:104CC4000090013602360336003600900136023673
:104CD4000336B60E0024F66E5B0E0120F76E000E4E
:104CE4000220F86E0900F5CF04F00900F5CF05F0B5
:104CF4000900F5CF06F00900F5CF07F0CBC000F0AE
:104D0400CCC001F0CDC002F0CEC003F0C7EC13F06C
:104D14000F0E0016000E011602160316120E0024C2
:104D2400F66E5C0E0120F76E000E0220F86E09008C
:104D3400F5CFC0F044D0BEC000F0BFC001F0000EFB
:104D4400BFBFFF0E026E036E0036009001360236BE
:104D5400033600360090013602360336B60E0024C0
:104D6400F66E5B0E0120F76E000E0220F86E09004D
:104D7400F5CF04F00900F5CF05F00900F5CF06F0F2
:104D84000900F5CF07F0CBC000F0CCC001F0CDC0D6
:104D940002F0CEC003F0C7EC13F00F0E0016000EA5
:104DA400011602160316230E0024F66E5C0E012073
:104DB400F76E000E0220F86E0900F5CFC0F047D060
:104DC400BEC000F0BFC001F0000EBFBFFF0E026EF8
:104DD400036E00360090013602360336003600902A
:104DE400013602360336CE0E0024F66E5A0E01202A
:104DF400F76E000E0220F86E0900F5CF04F00900EA
:104E0400F5CF05F00900F5CF06F00900F5CF07F05E
:104E1400CBC000F0CCC001F0CDC002F0CEC003F096
:104E2400C7EC13F0070E0014C06F300EC0270FD06C
:104E3400D151000AD8B4F2D6D151C00AD8B4EED6B2
:104E4400D151800AD8B430D7D151400AB9E0AFC0AB
:104E5400E1FFB0C0E2FFC0C0E6FFAF4BB02BCF4BC9
:104E6400D02BCAD6C3A71AD0800E006E800EC219EA
:104E7400005C02E1C151000811E2AFC0E1FFB0C023
:104E8400E2FF200EE66EAF4BB02BCF4BD02B010EC2
:104E9400C15F000EC25BC151C211EFE147EF17F0D1
:0A4EA400CFC000F0D0C001F01200F2
:104EAE0038EC0FF000C0AFF0FE0E0001D76F5A0EB7
:104EBE00D86F000ED96F20EC0EF000C0B0F0AF51DD
:104ECE00005C03E2AFC000F002D0B0C000F01200F0
:104EDE000001B56B200E385C03E36DB201D002D039
:104EEE00006A2FD080C0D7F081C0D8F097EC0FF0B9
:104EFE00005226E180C0B3F081C0B4F0000E8119DB
:104F0E0002E1000E80190AE0010EB325E96E000ED3
:104F1E00B421EA6EEECF00F000C0B5F0B2C0D7F00B
:104F2E00D86BAFC0D9F0B0C0DAF0B1C0DBF0ADECE9
:104F3E000FF000C080F001C081F0B5C000F001D0CC
:044F4E00006A1200E3
:104F52000B6A0350D8B4EFEF27F002500A6E028EAC
:104F62008E0E035E03AEF3EF27F0036C080E035CB4
:104F7200D8A0CEEF27F0036E013602C001F0026A1C
:104F8200080E035CD8A0CEEF27F0036E0136016A4B
:104F92000350D8A4D890D8EF27F00350D8B4D8EF54
:104FA20027F0D89002320132032ED2EF27F00BBC49
:104FB20001A0E5EF27F0D8A0E5EF27F0012AD8B449
:104FC200022A02BE02EF28F00AAE08EF28F0021E03
:104FD200011E012AD8B4022A08EF28F0026A016AE7
:104FE20008EF28F00B800BAE0CEF28F0026A0AAE35
:104FF2000CEF28F0FF0E026E016E0A3602320CEF41
:1050020028F0010E0C6E06EC07F00EEF28F0000EF1
:105012000C6E0EEF28F0FF0E0C6E0150006E025067
:04502200016E120009
:105026009D0E0001A56F000EA66F98C0AFF099C047
:10503600B0F09AC0B1F09BC0B2F09CC0B3F0A50E20
:10504600B46F000EB56F42EC17F000C0A3F001C0BC
:10505600A4F000509825E16E01509921E26EE66AAF
:0A506600A3C000F0A4C001F0120086
:1050700087C0AFF088C0B0F0400E0001B16F010EE4
:06508000B26F2DDF1200EB
:105086000900F5CFE6FF0006FBE10106F9E1120093
:105096003850010A07E16DBA05D0686A69806988E7
:1050A600020E386E68A406D069A404D0FB0E6816FA
:1050B600C2EC06F06DA203D004EC07F0DDD068A0C8
:1050C60019D069A017D0FEEC09F0040E386E200E38
:1050D6000401026F040E036F080E016F000E001527
:1050E600006E00C000F48C0E0011006E00C000F4CB
:1050F600FE0E681668A806D069A804D0D3EC07F09F
:10510600EF0E681668AC04D069AC02D0BF0E681604
:1051160068AA04D069AA02D063EC07F068A202D09C
:1051260069B26A6A040E385C03E204EC07F0A4D0A4
:1051360069A6A0D00001DE6B040EDE5DD8B09AD061
:1051460068A694D06CCF76F0F70E6816780E7615B2
:10515600016E0150000AD8A488D0FD0E7615016EA6
:10516600026AFF0E0216000E021802E1000E011876
:105176006DE17E0E7615016E01C003F00332039ECB
:1051860003C000F0000E016E0036009001360036B6
:1051960000900136000E0024026E040E0120036EFC
:1051A60002C06FF003C070F002C095F003C096F025
:1051B600040E9519006E00C095F002C0E9FF03C009
:1051C600EAFFEECF00F000C001F03C0E01160132FE
:1051D600019E0132019E01500D0A35E1020E6F2536
:1051E600E96E000E7021EA6EEECF01F0EECF02F00E
:1051F6000250040A02E1280E011822E1020E6F2570
:10520600E16E000E7021E26E200EE66E040EE66E72
:10521600DD6B080EDD5D14E2200EE16E040EE26E1B
:10522600DD51E126D8B0E22A280EE96E040EEA6EB8
:10523600DD51E926D8B0EA2AEECFE6FFDD2BE9D725
:10524600EEEC06F002D0CAEC06F00ED0FD0E761596
:10525600016E026AFF0E0216000E021802E1040E2B
:10526600011802E181EC07F000D001D003D0000163
:0A527600DE2B62D704EC07F01200F3
:105280009CC000F000019C07005228E098C0E9FF94
:1052900099C0EAFFEE50000A0CE098C0E9FF99C0FF
:1052A000EAFF9AC0D9FF9BC0DAFFEE50DE1801E199
:1052B0000FD098C0E9FF99C0EAFF9AC0D9FF9BC000
:1052C000DAFFDE50EE5C006E016A000E015A08D073
:1052D0000001984B992B9A4B9B2BD2D7006A016AFD
:0252E0001200BA
:1052E20098C002F099C003F002C000F003C001F0C0
:1052F200024A032A00C0E9FF01C0EAFFEE5201E0C0
:10530200F3D700019851025C006E99510358016E67
:0A531200010E005E000E015A1200A9
:10531C0098C0AFF099C0B0F09AC0B1F0010E000186
:08532C00B26FEFEC16F0120065
:1053340000019E51000805E3070E9F6F000EA06F49
:1053440012D09E51160805E2170EA16F000EA26F2F
:1053540006D09E51010FA16FA26B000EA223A1C023
:105364009FF0A2C0A0F09FC0A9F0A0C0AAF0A36BB8
:10537400A46B046A056A066A076A98C000F099C0BB
:1053840001F09AC002F09BC003F00AEC0BF0010E8E
:10539400D8B0000E006E005209E09CC0E1FF9DC031
:1053A400E2FF2D0EE66E9C4B9D2B9A7F98C004F075
:1053B40099C005F09AC006F09BC007F0006A016A24
:1053C400026A036A0AEC0BF0010ED8B0000E006EFC
:1053D400005237E0000E046E000E056E000E066EDD
:1053E4007F0E076E98C000F099C001F09AC002F0D9
:1053F4009BC003F00AEC0BF0010ED8B0000E006E57
:1054040000521FE098C000F099C001F09AC002F069
:105414009BC003F0000E046E000E056E200E066E97
:10542400820E076E68EC0AF000C098F001C099F093
:1054340002C09AF003C09BF0010EA35F000EA45BB0
:10544400C9D7000E046E000E056E200E066E820E85
:10545400076E98C000F099C001F09AC002F09BC09A
:1054640003F00AEC0BF0000ED8B0010E006E0052EF
:105474001EE0000E046E000E056E200E066E820EF7
:10548400076E98C000F099C001F09AC002F09BC06A
:1054940003F071EC0BF000C098F001C099F002C069
:1054A4009AF003C09BF00001A34BA42BCAD7A351CD
:1054B400A927A451AA23010EA56F000EA66F010E01
:1054C400006E000E016EBEEC16F000C0ABF001C021
:1054D400ACF002C0ADF003C0AEF0800EA619006EB1
:1054E400800EAA19005C02E1A951A55D1EE2000E1E
:1054F400046E000E056E200E066E820E076EABC0A3
:1055040000F0ACC001F0ADC002F0AEC003F071EC2D
:105514000BF000C0ABF001C0ACF002C0ADF003C0B2
:10552400AEF00001A54BA62BD8D7000E046E000EDA
:10553400056E000E066E800E076EABC000F0ACC0A8
:1055440001F0ADC002F0AEC003F071EC0BF098C0F6
:1055540004F099C005F09AC006F09BC007F0EBEC8C
:1055640007F000C098F001C099F002C09AF003C09F
:105574009BF0000E046E000E056E200E066E820E69
:10558400076E0AEC0BF0000ED8B0010E006E00524C
:105594000BE0000E0001986F000E996F000E9A6FD9
:1055A4007F0E9B6FA34BA42B0001800EA419006EE9
:1055B400800E005C02E1000EA35D38E29CC0E1FFB6
:1055C4009DC0E2FF300EE66E9C4B9D2B9CC0E1FF1C
:1055D4009DC0E2FF2E0EE66E9C4B9D2B800EAA19F9
:1055E400006E800E005C02E1000EA95D04E2A95188
:1055F400A35FAA51A45BFF0EA56FFF0EA66F800EDA
:10560400A419006E800EA619005C02E1A551A35DE9
:105614000DE29CC0E1FF9DC0E2FF300EE66E9C4BA4
:105624009D2B010EA55F000EA65BE9D7A56BA66BAB
:10563400800EA619006E800EAA19005C02E1A95121
:10564400A55D62E298C000F099C001F09AC002F032
:105654009BC003F07CDC00C0A7F001C0A8F0300EB2
:1056640000269CC0E1FF9DC0E2FF00C0E6FF9C4B0A
:105674009D2BA651A41902E1A351A51908E19CC0D0
:10568400E1FF9DC0E2FF2E0EE66E9C4B9D2BA7C052
:1056940000F0A8C001F0BEEC16F000C0ABF001C0F1
:1056A400ACF002C0ADF003C0AEF000C004F001C025
:1056B40005F002C006F003C007F098C000F099C0DE
:1056C40001F09AC002F09BC003F0FBEC0AF000C0AA
:1056D40098F001C099F002C09AF003C09BF0000E4C
:1056E400046E000E056E200E066E820E076E68ECC8
:1056F4000AF000C098F001C099F002C09AF003C00B
:105704009BF0A54BA62B94D79CC0E1FF9DC0E2FF64
:04571400E66A12002F
:1057180057EC27F000C082F0010E746F98C087F034
:1057280099C088F09AC072F09BC073F0FEEC09F043
:10573800010E016E0150010A02E1DFEC16F01200C1
:105748000050086E0150006E016A026A036A0B6A13
:105758000C6A960E036E0A6A00C001F008C000F0D9
:0A576800086A026A48EC0DF0120016
:1057720024EC2EF09280929293920A0E0B6E220EDD
:105782000C6EA10E0D6E0D2EFED70C2EFCD70B2E1D
:10579200FAD78A948A92070EB46EC26AC16AC19A13
:1057A200C198C186C184C182C190C08EC08AC0889E
:1057B200C086C084C084C094C280070E0B6E170ED0
:1057C2000C6E6A0E0D6E0D2EFED70C2EFCD70B2E14
:1057D200FAD70000080E0001976F000E986F050EB1
:1057E200996F400E9A6F050E9B6F95DF40DC005259
:1057F20001E1FCD7000E986F050E996F300E9A6F7B
:10580200000E9B6F030E9C6F3ADD000E011802E141
:10581200000E001862E1C294100E0C6E940E0D6E12
:105822000D2EFED70C2EFCD70000C282C2A201D0E0
:10583200FDD7C4CF03F0000E046E03C001F0006A6E
:10584200C3500012000E011200C068F001C069F0DE
:105852007ADF000E046E000E056E200E066E810EBB
:10586200076E68EC0AF0000E046E000E056E000E64
:10587200066E890E076E71EC0BF000C050F001C08D
:1058820051F002C052F003C053F000C098F001C0C2
:1058920099F002C09AF003C09BF0540E00019C6F75
:1058A200000E9D6F020E9E6F44DD400E986F050E36
:1058B200996F4F0E9A6F5B0E9B6F000E9C6F68C0C4
:1058C2009DF069C09EF068C09FF069C0A0F0540EC0
:1058D200A16F000EA26F13EC28F00001000E986F6A
:1058E200050E996F340E9A6F000E9B6F010E9C6F1E
:1058F200C6DC000E011802E1000E00182FE10001C3
:10590200972B0F0E9715016E01500A0A12E1060E2F
:105912009725006E016A000E0122600E046E000ED1
:10592200056ECFEC0EF008C000F009C001F000C017
:1059320097F0400E0001986F050E996FEB0E9A6F6B
:105942005B0E9B6F000E9C6F97C09DF0000E9E6FCA
:1059520097C09FF0000EA06F13EC28F00001000E1C
:10596200986F050E996F360E9A6F000E9B6F010E9F
:105972009C6F85DC000E011802E1000E001823E185
:10598200000197070F0E9715016E01500F0A02E1F1
:10599200060E975F9751590802E2590E976F400E13
:1059A200986F050E996FD60E9A6F5B0E9B6F000E65
:1059B2009C6F97C09DF0000E9E6F97C09FF0000EE7
:1059C200A06F13EC28F00001400E986F050E996F3E
:1059D20087DC00C06AF001C06BF00001400E986FD6
:1059E200050E996F400E9A6F98DC005201E1F5D7CF
:1059F20000016951030802E16851B60802E28A8493
:105A020001D08A94000E695D02E1320E685D02E205
:105A12008A8201D08A921F0E0B6E710E0C6E1E0EC0
:105A22000D6E0D2EFED70C2EFCD70B2EFAD70000D2
:045A3200DDD6FFD7E7
:105C480010EE29F00F0E006E010E016E340EF66E86
:0E5C58005C0EF76E000EF86E43EC28F01200A2
:105A36000000007F000020820000488500007A8870
:105A460000401C8C0050438F002474928096189658
:105A560020BC3E99286B6E9CF90215A0EC782DC1EE
:045A6600CAF249E255
:105A6A000000007FCDCC4C7B0AD723786F120375D8
:105A7A0017B75171ACC5276EBD37066B95BF566710
:105A8A0077CC2B645F700961FFE65B5D08E53C3CFF
:045A9A006042221B29
:105A9E0020035500530042002000480049004400F6
:105AAE0020004C00690062007200610072007900F3
:105ABE0000000000000000000000000000000000D8
:105ACE00010000000800000040000000000200007D
:105ADE000010000000800000000004000000200004
:105AEE00000000010000000800000040000000005F
:105AFE0009022900010100C032090400000203005E
:105B0E000000092101010001222100070581034047
:095B1E000001070501034000012C
:105B2700010000000A00000064000000E803000014
:105B370010270000A086010040420F0080969800C1
:085B470000E1F50500CA9A3BDC
:105B4F004144433D20252035752020202025303429
:105B5F00582020736F697420257320566F6C7473EF
:045B6F00200D0A00FB
:105B730022034D0069006B0072006F0065006C002A
:105B830065006B00740072006F006E0069006B00AB
:025B93006100AF
:105B95000600FF0901A10119012940150026FF0092
:105BA50075089540810219012940750895409102B3
:015BB500C02F
:105BB60001000000100000000001000000100000BD
:105BC60000000100000010000000000100000010AD
:105BD6007365633D2025336420202020253034580A
:055BE60020200D0A0063
:105BEB007365633D202533642020202025303458F5
:055BFB0020200D0A004E
:105C000012010002000000083412341201000102E7
:025C1000000191
:105C120030313233343536373839414243444546E0
:015C22000081
:105C2300303132333435363738396162636465660F
:015C33000070
:075C3400286E756C6C29005D
:045C3B00414443009D
:025C3F002B0038
:025C41002D0034
:045C43000403090449
:020000040030CA
:0E000000214E2E1EFF8181FF0FC00FE00F402A
:0200000400F00A
:1000000053544152545553422031384632353530DD
:100010005445535420555342205445524D494E4166
:100020004C202031302F30352F323031350D0A0041
:10003000FFFFFFFFFFFFFFFFFFFFFFFFFFFFFFFFD0
:10004000FFFFFFFFFFFFFFFFFFFFFFFFFFFFFFFFC0
:10005000FFFFFFFFFFFFFFFFFFFFFFFFFFFFFFFFB0
:10006000FFFFFFFFFFFFFFFFFFFFFFFFFFFFFFFFA0
:10007000FFFFFFFFFFFFFFFFFFFFFFFFFFFFFFFF90
:10008000FFFFFFFFFFFFFFFFFFFFFFFFFFFFFFFF80
:10009000FFFFFFFFFFFFFFFFFFFFFFFFFFFFFFFF70
:1000A000FFFFFFFFFFFFFFFFFFFFFFFFFFFFFFFF60
:1000B000FFFFFFFFFFFFFFFFFFFFFFFFFFFFFFFF50
:1000C000FFFFFFFFFFFFFFFFFFFFFFFFFFFFFFFF40
:1000D000FFFFFFFFFFFFFFFFFFFFFFFFFFFFFFFF30
:1000E000FFFFFFFFFFFFFFFFFFFFFFFFFFFFFFFF20
:1000F000FFFFFFFFFFFFFFFFFFFFFFFFFFFFFFFF10
:00000001FF
